:1000000016C3000033C3000031C300002FC300003B
:100010002DC300002BC3000029C3000027C300002C
:1000200025C3000023C3000021C300001FC300003C
:100030000C941A3D1BC3000019C3000017C3000035
:1000400015C3000013C300000C94063D0FC300004D
:100050000DC300000BC3000009C3000007C300006C
:1000600005C3000003C3000001C30000FFC200007D
:10007000FDC20000FBC20000F9C20000F7C2000090
:10008000F5C20000F3C20000F1C20000180A1D0A08
:100090002B0A300A350A3A0A3F0A440AD20DD70D14
:1000A000E50DEA0DEF0DF40DF90DFE0D531256128C
:1000B00059125C125F12621265126812A21EC71EEC
:1000C000DB1EEE1EF11E021F131F311FB81EBB1ECA
:1000D000241F271F2A1FBE1EC11EC41E3A245024DF
:1000E00064247C249224A824CC24E224F824C2266C
:1000F00019270F2866285C295E2A202BF22BF32C67
:100100002E2D822DC32DCC2D1C2E6C2E6F2E722EDB
:10011000752E782E7B2E7E2E812E2B31413157313C
:100120006E3184319A31B031C6311A321D322032EB
:100130002332263229322C322F32873203337F3357
:100140000834913408358435EE355836D1363E378B
:10015000B5373B38BE380000000000000000040442
:100160000404000400000A0A0A00000000000A0A51
:100170001F0A1F0A0A00040F140E051E0400181996
:100180000204081303000C12140814120D000C04CE
:100190000800000000000204080808040200080427
:1001A0000202020408000004150E150400000004F9
:1001B000041F04040000000000000C0408000000FC
:1001C000001F0000000000000000000C0C000001F7
:1001D0000204081000000E11131519110E00040C72
:1001E000040404040E000E11010204081F001F0283
:1001F000040201110E0002060A121F0202001F1063
:100200001E0101110E000608101E11110E001F0123
:100210000204080808000E11110E11110E000E1133
:10022000110F01020C000001020408100000000C74
:100230000C000C040800020408100804020000006E
:100240001F001F00000008040201020408000E1134
:100250000102040004000E11010D15150E000E110F
:1002600011111F1111001E11111E11111E000E116E
:10027000101010110E001C12111111121C001F1071
:10028000101E10101F001F10101E101010000E1155
:10029000101711110E001111111F111111000E0470
:1002A000040404040E000702020202120C001112E0
:1002B0001418141211001010101010101F00111B30
:1002C00015151111110011111915131111000E112D
:1002D000111111110E001E11111E101010000E111F
:1002E000111115120D001E11111E141211000F1004
:1002F000100E01011E001F04040404040400111167
:10030000111111110E0011111111110A0400111116
:10031000111115150E0011110A040A111100111105
:10032000110A040404001F01020408101F000E0833
:10033000080808080E00110A1F041F0404000E021A
:10034000020202020E00040A110000000000000078
:10035000000000001F000804000000000000000072
:100360000E010F110F0010101E1111111E000000C0
:100370000E1010110E0001010D1311110F000000DD
:100380000E111F100E000609081C08080800000FB7
:1003900011110F010E001010161911111100040097
:1003A0000C0404040E000200060202120C001010DD
:1003B0001214181412001808080808081C0000007D
:1003C0001A15151111000000161911111100000065
:1003D0000E1111110E0000001E111E101000000061
:1003E0000F110F010100000016191010100000007D
:1003F0000E100E011E0008081C0808090600000067
:10040000111111130D0000001111110A0400000058
:10041000111111150A000000110A040A1100000050
:1004200011110F010E0000001F0204081F003844C4
:1004300044447C4444007C40407844447800784400
:100440004478444478007C404040404040000C14D4
:10045000242424243C447C40407840407C00545474
:100460005438545454003844041804443800444464
:100470004C546444440054444C5464444400444840
:100480005060504844001C24242424246400446CFC
:100490005454444444004444447C44444400384458
:1004A0004444444438007C44444444444400784434
:1004B00044784040400038444040404438007C107C
:1004C0001010101010004444443C044438003854C8
:1004D0005454381010004444281028444400444424
:1004E000444444447E02444444443C040400545480
:1004F000545454547C005454545454547E02602038
:100500002038242438004444446454546400404057
:100510004078444478003844041C0444380048546B
:100520005474545448003C44443C14244400000097
:1005300038043C443C0000007840784478000000D7
:10054000784C784C78000000784040404000000033
:10055000182828287C44000038447C403C000000D7
:1005600054543854540000007804380478000000D3
:10057000444C546444000010444C54644400000053
:1005800044487048440000001C24444444000000D7
:10059000446C545444000000484878484800000027
:1005A0003844444438000000784848484800000077
:1005B0007048704040000000384040403800000063
:1005C0007C1010101000000048483808700000002F
:1005D000385454381000000044281028440000000B
:1005E000484848487C040000484838080800000093
:1005F000545454547C000000545454547E0200005F
:1006000060203C223C0000004242724A720000001E
:1006100040407844780000007008780870000000BE
:100620004C5272524C0000003C443C4444001124A3
:100630001FBECFEFD0E1DEBFCDBF15E0A0E0B1E03F
:10064000E8E6F6E800E00BBF02C007900D92A63D79
:10065000B107D9F726E0A6EDB5E001C01D92A63896
:10066000B207E1F70E94783D0C943243C9CCE2E630
:10067000F0E090819E7F9083908194609083908140
:10068000977F9083A8988BBB8DE08A95F1F7000047
:10069000A89A8081886080830895E2E6F0E09081E6
:1006A000916090839081946090839081977F9083F4
:1006B000A8988BBB8DE08A95F1F70000A89A8081FD
:1006C000886080830895CF93C82F892FE6DF8C2F11
:1006D000CF91E3CFE2E6F0E020812160208320810A
:1006E000246020832081277F2083A8988BBB92BB26
:1006F0008DE08A95F1F70000A89A80818860808358
:100700000895CF93C82F86E3B2DFC13049F030F0AF
:10071000C23041F0C33059F488EE07C088E403C00A
:1007200088E203C088E8B9DF04C0B7DF0BC0CD7F23
:1007300049F48FEE90E09093D9058093D8058FE32C
:1007400091E008C08FE391E09093D9058093D8059C
:100750008FEE90E09093D7058093D605CF910895C2
:10076000CF93C82F8FEF8ABB81BB8093610081E05C
:1007700084BBE2E6F0E080818260808381E077DF05
:100780002FEF89E698E1215080409040E1F700C0CA
:10079000000080EC6CDF85E280DF81EC68DF81E1C6
:1007A0007CDF85EC64DF8BE278DF8BE276DF87EC41
:1007B0005EDF86E872DF8C2FA4DF8AE358DF85E0F6
:1007C0006CDF81EB54DF80E068DF88E166DF86EB79
:1007D0004EDF8AE062DF82E860DF87E25EDF81E190
:1007E00046DF2FEF8DEE92E0215080409040E1F700
:1007F00000C0000089E2CF913ACF0F931F93CF93AF
:10080000DF938C01EB018AE232DFC8015CDFCE01AD
:10081000DF91CF911F910F9156CF0F931F93CF93DD
:10082000DF938C01EB018BE222DFC8014CDFCE01AC
:10083000DF91CF911F910F9146CFCF93DF93EB01C3
:10084000BC01DBDFBE01CE01E8DF8CE2DF91CF919E
:100850000ECFCF93DF93EA01F0DFCE01DF91CF918E
:1008600039CF8F929F92AF92BF92CF92DF92EF9249
:10087000FF920F931F93CF93DF93A8956817790783
:1008800038F4862797276827792786279727A895FA
:100890002417350738F442275327242735274227C2
:1008A0005327A895A091D805B091D905FC01A817A8
:1008B000B90708F4FD016B01A617B70708F46D012D
:1008C0008091D6059091D705EA018417950708F421
:1008D000EC0179018217930708F47C01A895960131
:1008E0002F5F3F4F2E1B3F0BD7011196AC1BBD0B4B
:1008F0000E94FA3F4B015C01B601CF017EDFA89553
:10090000B701CE018ADF8CE2B2DEA895C12CD12CD2
:100910007601C814D904EA04FB0449F0C801DADE00
:10092000A8958FEFC81AD80AE80AF80AF2CFDF9123
:10093000CF911F910F91FF90EF90DF90CF90BF90DC
:10094000AF909F908F9008950F931F93411551057D
:1009500079F02115310561F0FA01AB01615071099F
:10096000260F371FBC01615071096E0F7F1F79DFA1
:100970001F910F9108952F923F924F925F926F9225
:100980007F928F929F92AF92BF92CF92DF92EF921F
:10099000FF920F931F93CF93DF93CDB7DEB7679787
:1009A0000FB6F894DEBF0FBECDBF5C01798B688BAC
:1009B000598748873B872A870F83F12C28E0029FBD
:1009C000C00111241A821982E8E0F0E0FF8BEE8B5F
:1009D00047019C01285F31093B8B2A8BFC01E052C7
:1009E000F340FD8BEC8BC888D98889819A81C80E29
:1009F000D91E8A899B89EE89FF898E1B9F0B9C01DA
:100A00002A5A3E4F3F872E878C899D898E1B9F0BCC
:100A1000FC01EA5AFE4FFD87EC871E821D821C8274
:100A20001B8287E0682E712C412C512C212C312CFB
:100A3000FF81F7FD1EC0EE85FF85849190E0062CB6
:100A400002C0959587950A94E2F780FF08C0088553
:100A500019859701A701B6018D819E8107C00A857E
:100A60001B859701A701B6018B819C818A0D9B1D77
:100A700020C0FF81F03CF0F0EC85FD85849190E092
:100A8000062C02C0959587950A94E2F780FF09C06D
:100A9000088519859701A701B601C501820D931D2F
:100AA00008C00A851B859701A701B601C501840D01
:100AB000951D4ADF280C391C480C591CF1E06F1AAF
:100AC00071082B813C81280D391D3C832B838D813E
:100AD0009E81880D991D9E838D839FEF69167906EF
:100AE00009F0A6CFEE89FF893197FF8BEE8B298124
:100AF0003A812E0D3F1D3A832983EF2B09F073CFE6
:100B000067960FB6F894DEBF0FBECDBFDF91CF91D1
:100B10001F910F91FF90EF90DF90CF90BF90AF901B
:100B20009F908F907F906F905F904F903F902F900D
:100B300008954F925F926F927F928F929F92AF92A1
:100B4000BF92CF92DF92EF92FF920F931F93CF93BA
:100B5000DF93EC016B014A013901102F88E0089FF7
:100B6000500111242701F20101912F010023B1F05E
:100B70002091D8053091D905CE010896281739075C
:100B800020F4CA0CDB1CC1E0D0E0E12E9301A401EB
:100B9000B601CE01F0DECA0DDB1DE5CFDF91CF91AE
:100BA0001F910F91FF90EF90DF90CF90BF90AF908B
:100BB0009F908F907F906F905F904F9008956F926D
:100BC0007F928F929F92AF92BF92CF92DF92EF92DD
:100BD000FF920F93CF93DF9300D000D0CDB7DEB755
:100BE0006C015B014A013901C70119821A821B821B
:100BF0001C824AE0BE016F5F7F4F0E940940CE0118
:100C000001967C019301A401B501C60192DF0F900A
:100C10000F900F900F90DF91CF910F91FF90EF9079
:100C2000DF90CF90BF90AF909F908F907F906F900C
:100C300008950F931F932091D6053091D7056091A9
:100C4000D8057091D9058C0140E050E080E090E03B
:100C500008DE1F910F910895EF92FF920F931F935B
:100C6000CF93DF93EB018A017901BC01640F751FFB
:100C7000C4DDBE01CE01D1DD8CE2F9DCC0E0D0E004
:100C8000C017D10721F0C70125DD2196F9CFDF91EB
:100C9000CF911F910F91FF90EF900895EF92FF92E7
:100CA0000F931F93CF93DF93EB018A017901BC016E
:100CB000A4DDBE01600F711FCE01AFDD8CE2D7DC79
:100CC000C0E0D0E0C017D10721F0C70103DD2196B5
:100CD000F9CFDF91CF911F910F91FF90EF90089581
:100CE0002F923F924F925F926F927F928F929F923C
:100CF000AF92BF92CF92DF92EF92FF920F931F932A
:100D0000CF93DF9300D000D000D0CDB7DEB76C0119
:100D10007B015A0139012801261B370B3A832983AD
:100D20008A01081B190B17FF03C0119501951109C2
:100D3000CA14DB0420F022242A94322C03C022247B
:100D40002394312C89819A819E838D8397FF05C0DE
:100D50009195819591099E838D832D813E81319559
:100D6000219531093C832B83E614F70428F08FEF9B
:100D70009FEF9A83898304C021E030E03A8329837E
:100D800048018D819E81881A990AA201B701C60186
:100D900060DDC401880F991F2B813C818217930766
:100DA00064F0CA14DB0499F02D813E81821A930A03
:100DB000C20CD31C0817190744F3E614F70439F0E2
:100DC000800E911E89819A81E80EF91EDECF26964B
:100DD0000FB6F894DEBF0FBECDBFDF91CF911F914C
:100DE0000F91FF90EF90DF90CF90BF90AF909F90CA
:100DF0008F907F906F905F904F903F902F900895CD
:100E0000AF92BF92CF92DF92EF92FF920F931F9318
:100E1000CF93DF937C016B01EA01590198011CDF3C
:100E2000B501615071096C0D7D1D9801AE01C701BE
:100E300013DF9801A501B601C70130DFCE0101978C
:100E40009801A501B6018E0D9F1DDF91CF911F91D5
:100E50000F91FF90EF90DF90CF90BF90AF901ECF9B
:100E60002F923F924F925F926F927F928F929F92BA
:100E7000AF92BF92CF92DF92EF92FF920F931F93A8
:100E8000CF93DF931C012B01690150E0002711274C
:100E9000041B150BC1E0D0E0C41BD50BCC0FDD1F2C
:100EA000E12CF12CA6015701A40CB51CB5013101B0
:100EB000601A710AC301CDDCA601B5014801820C9C
:100EC000931CC401C6DCA6015201AE18BF08B501CF
:100ED000C401BFDCA601B501C301BBDCEC16FD06F5
:100EE000B4F08FEFE81AF80AC701880F991F01962E
:100EF0008C0F9D1F22273327201B310BE216F30690
:100F000039F40C171D074CF0C0E0D0E001C0CE0151
:100F10000C171D0714F0EC01C5CF0F5F1F4F980190
:100F2000220F331F2F5F3F4F820F931F10161106A2
:100F300094F7DF91CF911F910F91FF90EF90DF9089
:100F4000CF90BF90AF909F908F907F906F905F9069
:100F50004F903F902F9008954F925F926F927F92A3
:100F60008F929F92AF92BF92CF92DF92EF92FF92B9
:100F70000F931F93CF93DF93EC015B014A0139017B
:100F800028018601ADDE9701A201B301C401A8DEEC
:100F90009501AE01B701C201A3DEDF91CF911F9190
:100FA0000F91FF90EF90DF90CF90BF90AF909F9008
:100FB0008F907F906F905F904F900895CF93C82F40
:100FC0008A3011F48DE0FADF5D9BFECFCCB980E072
:100FD00090E0CF910895CF92DF92EF92FF920F931E
:100FE0001F93A8950FEF1FEF21E430E04FE550E08D
:100FF00065E070E085E090E003DFA89521E430E053
:101000004FE550E06BE470E085E090E0F9DE2BE422
:1010100030E04FE550E061E970E085E090E0F0DE1F
:10102000A3E2EA2EA5E0FA2E01E02FE130E04FEF37
:101030005FEF60E570E082E190E07BDDBEE1EB2EEA
:10104000B5E0FB2E2FE130E04FEF5FEF6AE570E097
:1010500083E290E06EDD0FEF1FEF21E430E04FE51B
:1010600050E065E070E08CED90E0CADE21E430E015
:101070004FE550E06BE470E08CED90E0C1DE2BE4D6
:1010800030E04FE550E061E970E08CED90E0B8DED3
:1010900013E2E12E15E0F12E01E02FE130E04FEFF9
:1010A0005FEF60E570E08BEE90E043DD88E1E82ED5
:1010B00085E0F82E2FE130E04FEF5FEF6AE570E05A
:1010C0008CEF90E036DD99E4E92E92E0F92E2FE1E5
:1010D00030E04FEF5FEF66EE70E08AE090E029DDF0
:1010E000A8958091120690911306019709F04FC0C0
:1010F0000FE110E024E430E048E550E064E970E0FE
:1011000088E090E021DC2CE430E04EE650E06CE832
:1011100070E089E690E018DC24E430E048E550E037
:1011200064E970E080EE90E00FDC20EE37E048E20A
:1011300064EB70E080EA90E093DE20EE37E047E277
:1011400064EB70E080EA90E08BDE20EE37E04BE26B
:1011500064EB70E080EA90E083DE20EE37E045E269
:1011600064EB70E080EA90E07BDEE0EECE2EE7E01C
:10117000DE2EF4EBEF2EF12C07EB10E028EC30E044
:1011800044E950E060EA70E084E990E0E5DEA8958B
:101190008091120690911306892B09F051C00FE13E
:1011A00010E024E430E048E550E064E970E088E0D5
:1011B00090E0CADB2CE430E04EE650E06CE870E0F2
:1011C00089E690E0C1DB24E430E048E550E064E9E2
:1011D00070E080EE90E0B8DB20E038EF48E264EBAE
:1011E00070E080EA90E03CDE20E038EF47E264EB1C
:1011F00070E080EA90E034DE20E038EF4BE264EB10
:1012000070E080EA90E02CDE20E038EF45E264EB0D
:1012100070E080EA90E024DE00E018EF23E230E0A6
:1012200045E050E065EA70E086E990E08DDB23E27E
:1012300030E045E050E065EA70E085EA90E084DB6C
:10124000A8958091140690911506892B79F4A8959C
:101250007EE0E72E75E0F72E01E02FE130E04FEF62
:101260005FEF63E270E08AE090E063DC8091140657
:10127000909115060197E1F4A89557ECE52E55E0FD
:10128000F52E01E02FE130E04FEF5FEF64E170E019
:1012900084E190E04EDC61ECE62E65E0F62E2FE175
:1012A00030E04FEF5FEF68E270E08EE190E041DC0C
:1012B000A89580911406909115060297E1F4A895DF
:1012C0003AEBE32E35E0F32E01E02FE130E04FEF73
:1012D0005FEF64E170E084E190E02BDC41ECE42E10
:1012E00045E0F42E2FE130E04FEF5FEF68E270E071
:1012F0008EE190E01EDCA895809114069091150671
:10130000039779F4A89523EBE22E25E0F22E01E075
:101310002FE130E04FEF5FEF63E270E089E190E0B2
:1013200008DCA8958091140690911506049779F42D
:10133000A89594EDE92E94E0F92E01E02FE130E03C
:101340004FEF5FEF63E270E08FE090E0F2DBA89593
:1013500080911406909115060597E1F4A8950EEC7E
:10136000E02E04E0F02E01E02FE130E04FEF5FEFE0
:1013700064E170E089E190E0DCDB84ECE82E84E05D
:10138000F82E2FE130E04FEF5FEF63E270E08FE087
:1013900090E0CFDBA89580911406909115060697F2
:1013A000E1F4A895BEECEB2EB4E0FB2E01E02FE1BA
:1013B00030E04FEF5FEF64E170E089E190E0B9DB8E
:1013C00012EBE12E14E0F12E2FE130E04FEF5FEF52
:1013D00063E270E08FE190E0ACDBA89580911406A9
:1013E00090911506079779F4A895A9E9EA2EA4E04B
:1013F000FA2E01E02FE130E04FEF5FEF63E270E0A3
:101400008FE090E096DB8091140690911506892B71
:1014100009F048C0A895E09171068E2F90E08830C1
:10142000910508F03FC0FC01EA5BFF4F0C94F13FCF
:10143000F4E9EF2EF4E0FF2E04C0EFE8EE2EE4E036
:10144000FE2E02E02FE130E04FEF5FEF6EE170E043
:101450008BEE90E026C075E8E72E74E0F72E18C0FA
:101460006BE7E62E64E0F62E13C051E7E52E54E05C
:10147000F52E0EC047E6E42E44E0F42E09C03DE50B
:10148000E32E34E0F32E04C023E5E22E24E0F22E16
:1014900001E02FE130E04FEF5FEF6EE170E086EEAC
:1014A00090E047DB8091140690911506019701F5B5
:1014B000A89580911D06813069F038F08230C1F422
:1014C00001E7E02E04E0F02E09C095E8E92E94E053
:1014D000F92E04C08BE7E82E84E0F82E01E02FE11E
:1014E00030E04FEF5FEF6EE170E086EE90E021DBE1
:1014F0008091140690911506029701F5A8958091A8
:101500002406813069F038F08230C1F4A1E7EA2E78
:10151000A4E0FA2E09C015E8E12E14E0F12E04C073
:10152000BBE7EB2EB4E0FB2E01E02FE130E04FEF04
:101530005FEF6EE170E086EE90E0FBDA80911406DA
:1015400090911506039779F4A895FFEDEF2EF4E03E
:10155000FF2E01E02FE130E04FEF5FEF6EE170E032
:101560008EEE90E0E6DA80911406909115060497CD
:1015700001F5A89580917C06813069F038F08230C1
:10158000C1F461E7E62E64E0F62E09C0E5E8EE2E30
:10159000E4E0FE2E04C07BE7E72E74E0F72E01E0C6
:1015A0002FE130E04FEF5FEF6EE170E086EE90E00C
:1015B000C0DA8091140690911506059701F5A8955B
:1015C00080917006813069F038F08230C1F431E7E3
:1015D000E32E34E0F32E09C055E8E52E54E0F52E55
:1015E00004C04BE7E42E44E0F42E01E02FE130E0AC
:1015F0004FEF5FEF6EE170E086EE90E09ADA809157
:10160000140690911506069701F5A89580916D0630
:10161000813069F038F08230C1F481E7E82E84E04F
:10162000F82E09C025E8E22E24E0F22E04C09BE744
:10163000E92E94E0F92E01E02FE130E04FEF5FEF6B
:101640006EE170E086EE90E074DA8091140690917D
:101650001506079709F4A8951F910F91FF90EF9039
:10166000DF90CF900895CF92DF92EF92FF920F9389
:101670001F93A89500EE17E021E430E048EC50E01D
:101680006AEA70E085E090E05FD90FEF1FEF21E498
:1016900030E048EC50E063E270E085E090E0B0DBE1
:1016A00087E6E82E82E0F82E01E02FE130E040EE00
:1016B00057E06CE370E088E290E03BDA0FEF1FEF59
:1016C00020E530E040E550E065E070E08BEE90E032
:1016D00097DB90EEC92E97E0D92E24E1E22EF12C73
:1016E00003E111E026E430E041E351E066E470E01C
:1016F00085EF90E031DC37E1E32EF12C24E430E09B
:101700004FE251E064E470E087EF90E025DC0FEFFA
:101710001FEF20E530E040E550E064E670E08BEE3E
:1017200090E06EDB45EAE42EF12C03E111E023E7C3
:1017300030E041E351E063E770E085EF90E00CDCDE
:1017400053EAE52EF12C25E730E04FE251E065E762
:1017500070E087EF90E000DC66E3E62E65E0F62EB1
:1017600002E020EE37E040E050E068EC70E08DE20F
:1017700090E0DFD91F910F91FF90EF90DF90CF9015
:101780000895CF92DF92EF92FF920F931F93A89547
:1017900000EE17E021E430E048EC50E06AEA70E047
:1017A00085E090E0D1D80FEF1FEF21E430E048EC66
:1017B00050E063E270E085E090E022DB83EAE82E0F
:1017C00084E0F82E01E02FE130E040EE57E06CE3DA
:1017D00070E088E290E0ADD90FEF1FEF20E530E038
:1017E00040E550E065E070E08BEE90E009DB90EEC4
:1017F000C92E97E0D92E24E1E22EF12C03E111E06D
:1018000026E430E041E351E066E470E085EF90E0EB
:10181000A3DB37E1E32EF12C24E430E04FE251E08A
:1018200064E470E087EF90E097DB0FEF1FEF20E5B7
:1018300030E040E550E064E670E08BEE90E0E0DA06
:1018400045EAE42EF12C03E111E023E730E041E327
:1018500051E063E770E085EF90E07EDB53EAE52E30
:10186000F12C25E730E04FE251E065E770E087EFCB
:1018700090E072DB6FECE62E65E0F62E02E020EEE3
:1018800037E040E050E068EC70E08DE290E051D944
:101890001F910F91FF90EF90DF90CF900895CF921E
:1018A000DF92EF92FF920F931F93A89500EE17E03F
:1018B00021E430E048EC50E06AEA70E085E090E036
:1018C00043D80FEF1FEF21E430E048EC50E063E233
:1018D00070E085E090E094DA82E4E82E84E0F82E6F
:1018E00001E02FE130E040EE57E06CE370E088E289
:1018F00090E01FD90FEF1FEF20E530E040E550E00A
:1019000065E070E08BEE90E07BDA90EEC92E97E018
:10191000D92E24E1E22EF12C03E111E026E430E09F
:1019200041E351E066E470E085EF90E015DB37E1DC
:10193000E32EF12C24E430E04FE251E064E470E067
:1019400087EF90E009DB0FEF1FEF20E530E040E587
:1019500050E064E670E08BEE90E052DA45EAE42E67
:10196000F12C03E111E023E730E041E351E063E7CC
:1019700070E085EF90E0F0DA53EAE52EF12C25E7F0
:1019800030E04FE251E065E770E087EF90E0E4DAA5
:1019900067E4E62E65E0F62E02E020EE37E040E058
:1019A00050E068EC70E08DE290E0C3D81F910F9199
:1019B000FF90EF90DF90CF900895CF93DF9300D00A
:1019C00000D0CDB7DEB7809163001C821B821A82E3
:1019D0001982BE016F5F7F4FCE0103960E94543E75
:1019E0008B819C818431954068F489819A81843A05
:1019F000964040F489819A818D32914018F082E0BE
:101A000080933A068B819C818937954090F08B8139
:101A10009C81843C994068F489819A81843A9640FB
:101A200040F489819A818D32914018F083E080934F
:101A30003A068B819C8189329A4068F089819A812B
:101A400084379E4040F489819A81813D974018F007
:101A500081E080933A068B819C81863F994060F4B7
:101A60008B819C818134964038F089819A81813DB7
:101A7000974010F010923A0680913A060F900F901E
:101A80000F900F90DF91CF910895CF92DF92EF9258
:101A9000FF920F931F93A89500EE17E021E430E02A
:101AA00048EC50E06AEA70E085E090E00E94A4040F
:101AB0000FEF1FEF21E430E048EC50E063E270E00C
:101AC00085E090E09DD920E530E040E550E065E01C
:101AD00070E08BEE90E094D9F0EECF2EF7E0DF2EA1
:101AE000A4E1EA2EF12C03E111E026E430E041E329
:101AF00051E066E470E085EF90E02EDAB7E1EB2E7E
:101B0000F12C24E430E04FE251E064E470E087EF30
:101B100090E022DA0FEF1FEF20E530E040E550E0E3
:101B200064E670E08BEE90E06BD915EAE12EF12CC3
:101B300003E111E023E730E041E351E063E770E0C7
:101B400085EF90E009DA83EAE82EF12C25E730E012
:101B50004FE251E065E770E087EF90E0FDD99FEC40
:101B6000E92E95E0F92E02E020EE37E040E050E06B
:101B700068EC70E08CE390E00E9499058091140677
:101B800090911506892B09F048C0E09171068E2FBF
:101B900090E08830910508F040C0FC01E25BFF4F07
:101BA0000C94F13FE4E9EE2EE4E0FE2E04C07FE861
:101BB000E72E74E0F72E02E02FE130E04FEF5FEF09
:101BC00065E070E086E490E026C065E8E62E64E01B
:101BD000F62E18C05BE7E52E54E0F52E13C041E762
:101BE000E42E44E0F42E0EC037E6E32E34E0F32E6C
:101BF00009C02DE5E22E24E0F22E04C093E5E92E83
:101C000094E0F92E02E02FE130E04FEF5FEF65E066
:101C100070E08EE190E00E94990580911406909109
:101C20001506019701F580911D06813069F038F0A5
:101C30008230C9F411E7E12E14E0F12E09C085E8E5
:101C4000E82E84E0F82E04C00BE7E02E04E0F02E2E
:101C500002E02FE130E04FEF5FEF65E070E08EE1F2
:101C600090E00E94990580911406909115060297C4
:101C700001F580912406813069F038F08230C9F492
:101C8000F1E7EF2EF4E0FF2E09C0B5E8EB2EB4E04B
:101C9000FB2E04C0ABE7EA2EA4E0FA2E02E02FE10F
:101CA00030E04FEF5FEF65E070E08EE190E00E9482
:101CB00099058091140690911506049701F580917D
:101CC0007C06813069F038F08230C9F461E7E62E95
:101CD00064E0F62E09C0E5E8EE2EE4E0FE2E04C036
:101CE0007BE7E72E74E0F72E02E02FE130E04FEFC4
:101CF0005FEF65E070E08EE190E00E9499058091D1
:101D0000140690911506059701F5809170068130B3
:101D100069F038F08230C9F431E7E32E34E0F32E75
:101D200009C055E8E52E54E0F52E04C04BE7E42E3B
:101D300044E0F42E02E02FE130E04FEF5FEF65E08A
:101D400070E08EE190E00E949905809114069091D8
:101D50001506069701F580916D06813069F038F01F
:101D60008230C9F481E7E82E84E0F82E09C025E826
:101D7000E22E24E0F22E04C09BE7E92E94E0F92E37
:101D800002E02FE130E04FEF5FEF65E070E08EE1C1
:101D900090E00E9499051F910F91FF90EF90DF90C6
:101DA000CF900895EF92FF920F931F9380910B06AF
:101DB00090910C060A97A8F48091E20581110CC05D
:101DC0000FE110E02CE330E044E650E06BE470E01B
:101DD0008EE690E00E94A40481E08093E2051092D8
:101DE000160680910B0690910C060A978A3591058C
:101DF000A8F48091160681110CC00FE110E02CE3CD
:101E000030E044E650E06BE470E08EE690E00E9443
:101E1000A40481E0809316061092E20580910B06DF
:101E200090910C0684369105A0F0809116068130C1
:101E300061F40FE110E02CE330E044E650E06BE4A5
:101E400070E08EE690E00E94A404109216061092B4
:101E5000E2058091120690911306019779F4E090C3
:101E60000B06F0900C0603E02FE130E04FEF5FEF40
:101E700064E670E082E890E00E94DF05809112063F
:101E800090911306892B79F4E0900B06F0900C06E4
:101E900003E02FE130E040E058EF64E670E082E8D4
:101EA00090E00E94DF051F910F91FF90EF90089541
:101EB000EF92FF920F931F9380913E0690913F0601
:101EC0000A97A8F480910A06811111C00FE110E071
:101ED00027E330E048E550E06BE970E088E090E00F
:101EE0000E94A40481E080930A0610926E068091FD
:101EF0003E0690913F0684369105D8F480910B06FA
:101F000090910C060A97A8F080916E06811111C07D
:101F10000FE110E027E330E048E550E06BE970E0C6
:101F200088E090E00E94A40481E080936E06109205
:101F30000A0680913E0690913F0684369105A0F0F6
:101F400080916E06813061F40FE110E027E330E00C
:101F500048E550E06BE970E088E090E00E94A4045E
:101F600010926E0610920A06E0903E06F0903F0630
:101F700003E02FE130E04FEF5FEF64EB70E08FE0C4
:101F800090E00E94DF051F910F91FF90EF90089560
:101F9000EF92FF920F931F9380912B0690912C0646
:101FA0000A97A8F48091110681110CC00FE110E08E
:101FB00024E230E04AE550E064E670E088E090E03A
:101FC0000E94A40481E0809311061092280680915B
:101FD0002B0690912C060A978A359105A8F48091DA
:101FE000280681110CC00FE110E024E230E04AE540
:101FF00050E064E670E088E090E00E94A40481E094
:10200000809328061092110680912B0690912C0641
:1020100084369105A1F480912806813061F40FE1A6
:1020200010E024E230E04AE550E064E670E088E049
:1020300090E00E94A404109211061092280680914C
:102040002B0690912C068436910530F084E690E0C2
:1020500090932C0680932B06E0902B06F0902C0694
:1020600003E02FE130E04FEF5FEF6EE670E084E1D8
:1020700090E00E94DF0580917D0690917E060A9790
:10208000A8F480917706811111C00FE110E024E2DD
:1020900030E04AE550E064E670E08FED90E00E94A9
:1020A000A40481E0809377061092400680917D061B
:1020B00090917E060A978A359105A8F48091400692
:1020C000811111C00FE110E024E230E04AE550E058
:1020D00064E670E08FED90E00E94A40481E08093BC
:1020E00040061092770680917D0690917E06843698
:1020F000910529F4109277061092400603C08436A9
:10210000910530F084E690E090937E0680937D0602
:10211000E0907D06F0907E0603E02FE130E04FEF87
:102120005FEF6EE670E089EE90E00E94DF051F91A0
:102130000F91FF90EF900895CF93DF9300D000D0E0
:10214000CDB7DEB7809163001C821B821A82198290
:10215000BE016F5F7F4FCE0103960E94543E8B817C
:102160009C81853C9940A0F0A89589819A81843C06
:10217000994070F4A89589819A818D3D954040F0F1
:10218000A89581E090E09093130680931206A8959D
:102190000F900F900F900F90DF91CF910895CF93F4
:1021A000DF9300D000D0CDB7DEB7A8958091630053
:1021B0001C821B821A821982BE016F5F7F4FCE0183
:1021C00003960E94543E8B819C81853C9940A8F0E7
:1021D00089819A81843C994080F489819A818D3DDE
:1021E000954058F010921306109212068FE19EE46B
:1021F0000197F1F700C00000A8950F900F900F9085
:102200000F90DF91CF9108957F928F929F92AF921E
:10221000BF92CF92DF92EF92FF920F931F93CF93D3
:10222000DF93EC016B015A014901702EA895809152
:10223000E5059091E6050A97A8F480917206811150
:1022400011C00FE110E02EE130E044E650E06550AF
:102250007109CE0144970E94A40481E08093720624
:10226000109233068091E5059091E6050A978A352C
:102270009105C0F480913306811114C00FE110E084
:102280002EE130E044E650E0B60165507109CE0120
:1022900044970E94A40481E0809333061092720652
:1022A00010920D068091E5059091E6058436910522
:1022B000C0F080910D06811114C00FE110E02EE1F5
:1022C00030E044E650E0B60165507109CE01449714
:1022D0000E94A40481E080930D06109233061092B0
:1022E0007206E090E505F090E605072D9401A50142
:1022F000B601CE010E94DF05A895DF91CF911F9115
:102300000F91FF90EF90DF90CF90BF90AF909F9094
:102310008F907F900895A89580913006813071F458
:10232000A49A80E185BBA8952FEF82E597E0215024
:1023300080409040E1F700C0000015BAA8950895CC
:10234000A89580913006813021F5A49A80E185BB63
:102350002FEF32E597E0215030409040E1F700C088
:102360000000A89515BA2FEF32E597E021503040D4
:102370009040E1F700C00000A89585BB2FEF32E543
:1023800087E0215030408040E1F700C00000A89570
:1023900015BA0895A89580913006813009F048C09B
:1023A000A49A80E185BBA8952FEF32E597E02150F4
:1023B00030409040E1F700C00000A89515BAA895FC
:1023C0002FEF32E597E0215030409040E1F700C018
:1023D0000000A89585BBA8952FEF32E597E0215026
:1023E00030409040E1F700C00000A89515BAA895CC
:1023F0002FEF32E597E0215030409040E1F700C0E8
:102400000000A89585BB2FEF32E587E021503040D2
:102410008040E1F700C00000A89515BA9FEF22E5C3
:1024200037E0915020403040E1F700C00000A8950F
:102430000895A89510922D06109221061092E0059D
:102440001092430610921E061092100610922F064C
:102450001092270610923D061092E10583EB92E060
:102460000E940C4380933006A89584EB92E00E9472
:1024700014439093230680932206A8958091140616
:1024800090911506892B51F5A895E09171068E2F34
:1024900090E08830910510F5FC01EA5AFF4F4EE1BB
:1024A00050E00C94F13F64E972E014C066E772E01A
:1024B00011C068E572E00EC06AE372E00BC06CE127
:1024C00072E008C06EEF71E005C060EE71E002C01E
:1024D00062EC71E08BEE95E00E94FC42A895809141
:1024E0001406909115060197D1F4A89580911D06C8
:1024F000813069F038F0823091F44EE150E068E6C6
:1025000071E009C04EE150E064EA71E004C04EE1C0
:1025100050E066E871E08BEE95E00E94FC42A895E1
:1025200080911406909115060297D1F4A895809198
:102530002406813069F038F0823091F44EE150E0A9
:102540006EE071E009C04EE150E06AE471E004C061
:102550004EE150E06CE271E08BEE95E00E94FC42AF
:10256000A89580911406909115060497C9F480915E
:102570007C06813069F038F0823091F44EE150E011
:1025800064EB70E009C04EE150E060EF70E004C021
:102590004EE150E062ED70E08BEE95E00E94FC426F
:1025A000A89580911406909115060597C9F480911D
:1025B0007006813069F038F0823091F44EE150E0DD
:1025C0006AE570E009C04EE150E066E970E004C0E1
:1025D0004EE150E068E770E08BEE95E00E94FC422F
:1025E000A89580911406909115060697C9F48091DC
:1025F0006D06813069F038F0823091F44EE150E0A0
:1026000060E070E009C04EE150E06CE370E004C0AF
:102610004EE150E06EE170E08BEE95E00E94FC42EE
:10262000A89587EC90E00197F1F700C00000809139
:10263000EB059091EC059093DF058093DE0580918A
:10264000ED059091EE0590933206809331068091CE
:10265000EF059091F00590937A068093790680912A
:10266000F1059091F20590931C0680931B068091D2
:10267000F305809346068091F5059091F6059093B9
:102680001A06809319068091F70580932A06809197
:10269000F905809329068091FB058093DA058091E6
:1026A000FD059091FE0590936A06809369068091DE
:1026B000FF05909100069093450680934406809113
:1026C000140690911506079741F4809101069091A8
:1026D000020690931506809314068091030690914C
:1026E0000406909368068093670680910506909192
:1026F00006069093EA058093E9058091070690917C
:10270000080690930F0680930E06A89508951092E0
:102710007E0610927D06BC9A80917D06880F81BF4F
:1027200010922C0610922B06139A80912B06880F7C
:10273000809386002FDE8DE490E090937406809362
:10274000730681E090E0909313068093120608953B
:10275000CF934091E5055091E60520911B063091FD
:102760001C06429FC001439F900D529F900D112463
:102770006AE070E00E94DD3F70934206609341067C
:1027800080912B0690912C068536910530F084E6D9
:1027900090E090932C0680932B068091290690E080
:1027A00020912B0630912C068217930720F49093EA
:1027B0002C0680932B0620912D06211114C0209108
:1027C0003E0630913F062233310538F424E630E0EE
:1027D00030932C0620932B0606C02233310519F0C6
:1027E00021E020932D0620912D0640913106509135
:1027F00032062130E1F520912B0630912C0624364B
:10280000310530F024E630E030932C0620932B067F
:102810006417750760F5E0913E06F0913F06209140
:102820002B0630912C06E617F707C0F42F5F3F4FB9
:102830008217930728F030932C0620932B0604C0B0
:1028400090932C0680932B0620912B0630912C061A
:102850002536310560F024E630E005C0211531054C
:1028600031F02150310930932C0620932B06461766
:10287000570708F04AC020913E0630913F062417C2
:102880003507D0F460912B0670912C066F5F7F4F57
:102890006536710510F064E670E070932C06609365
:1028A0002B0660912B0670912C068617970720F453
:1028B00090932C0680932B064217530730F5809196
:1028C0002B0690912C06009729F0019790932C06E7
:1028D00080932B06241B350B2B303105B0F08091F3
:1028E0002B0690912C060A9720F410922C06109239
:1028F0002B0680912B0690912C068A30910528F0AA
:102900000A9790932C0680932B06C0914606C130FF
:10291000D1F480912106811116C020910B063091CF
:102920000C068091190690911A062817390759F458
:1029300080913E0690913F06909332068093310637
:10294000EADCC0932106C091DA05C13009F5809117
:10295000E00581111DC080910B0690910C0620911D
:10296000690630916A06821B930B059788F42091C3
:102970003106309132068091440690914506820FCF
:10298000931F9093320680933106C5DCC093E00517
:10299000CF9108958091430681111CC080910B0650
:1029A00090910C062091190630911A06821B930B08
:1029B000029780F482E390E090937E0680937D06F8
:1029C00081E0809343068093100680914606811132
:1029D00001C0A1DC2091190630911A06609175069C
:1029E000709176064091790650917A06649FC001F5
:1029F000659F900D749F900D11246AE070E00E9415
:102A0000DD3F620F731F7093DD056093DC05E0917D
:102A10007D06F0917E064091DE055091DF05461758
:102A2000570720F45093DD054093DC0580912A067A
:102A300090E08E179F0720F490937E0680937D068A
:102A400080910B0690910C062817390720F0481743
:102A50005907A0F176C020913D062111F8CF8417C7
:102A60009507A8F76091DC057091DD0520917D0642
:102A700030917E068617970788F42F5F3F4F2536E3
:102A8000310528F430937E0620937D06E0CF24E6BE
:102A900030E030937E0620937D06A6C021153105D7
:102AA00031F02150310930937E0620937D0620912C
:102AB0007D0630917E06232B51F296C020917D0633
:102AC00030917E062115310531F0215031093093C6
:102AD0007E0620937D06841B950B0697B0F08091AF
:102AE0007D0690917E060A9720F410927E06109241
:102AF0007D0680917D0690917E068A30910528F0B2
:102B00000A9790937E0680937D068091E10581115E
:102B100006C016DC81E0809327068093E1052091B2
:102B2000E7053091E80580912206909123068217EF
:102B3000930738F4ECDD81E090E0909313068093E6
:102B4000120680911E06811158C04091670650916F
:102B500068068091190690911A068417950708F067
:102B60004CC0E0910B06F0910C064E175F0729F45C
:102B700081E080933D0680932F0680913D06813051
:102B8000E1F56091E3057091E4052091E90530914C
:102B9000EA0562177307A8F480917D0690917E067E
:102BA000E417F50738F401968536910530F084E690
:102BB00090E003C0009729F0019790937E068093E0
:102BC0007D0626173707C8F410923D0680917506DA
:102BD00090917606821B930B9093760680937506F0
:102BE00081E080931E0608954817590708F0A9CF81
:102BF00020917D0630917E0668CF0895809143062E
:102C000081111BC020910B0630910C068091190692
:102C100090911A068217930780F482E390E09093D4
:102C20007E0680937D0681E08093430680931006A4
:102C300080914606811101C06EDBE0911906F0918A
:102C40001A064091750650917606209179063091CA
:102C50007A06429FC001439F900D529F900D112410
:102C60006AE070E00E94DD3F6E0F7F1F7093DD050C
:102C70006093DC0520917D0630917E064091DE0553
:102C80005091DF054617570720F45093DD05409318
:102C9000DC0580912A0690E08217930720F4909338
:102CA0007E0680937D0620910B0630910C06E2177C
:102CB000F30700F580913D0681111CC024173507EC
:102CC000C8F46091DC057091DD0580917D069091DE
:102CD0007E062617370738F401968536910530F0C1
:102CE00084E690E003C0009729F0019790937E0658
:102CF00080937D0642175307E0F580917D06909101
:102D00007E06019790937E0680937D06241B350BEB
:102D10002630310590F00A9720F410927E0610922A
:102D20007D0680917D0690917E068A30910528F07F
:102D30000A9790937E0680937D068091E10581112C
:102D400006C0FEDA81E0809327068093E10520919A
:102D5000E7053091E80580912206909123068217BD
:102D6000930738F4D4DC81E090E0909313068093CD
:102D7000120680911E0681114EC040916706509147
:102D800068068091190690911A068417950708F035
:102D900042C0E0910B06F0910C064E175F0729F434
:102DA00081E080933D0680932F0680913D0681301F
:102DB00091F56091E3057091E4052091E90530916A
:102DC000EA0562177307A8F480917D0690917E064C
:102DD000E417F50738F401968536910530F084E65E
:102DE00090E003C0009729F0019790937E068093AE
:102DF0007D062617370778F410923D0680917506F8
:102E000090917606821B930B9093760680937506BD
:102E100081E080931E060895CF93C0914606C1308D
:102E2000D1F480912106811116C020910B063091BA
:102E30000C068091190690911A062817390759F443
:102E400080913E0690913F06909332068093310622
:102E500062DAC09321064091E5055091E605209184
:102E60001B0630911C06429FC001439F900D529F4C
:102E7000900D11246AE070E00E94DD3F70934206DD
:102E80006093410680912B0690912C068536910522
:102E900030F084E690E090932C0680932B0680918E
:102EA000290690E020912B0630912C06821793077B
:102EB00020F490932C0680932B0620912D0621114F
:102EC00014C020913E0630913F062639310538F472
:102ED00024E630E030932C0620932B0606C02639DA
:102EE000310519F021E020932D0620912D06409107
:102EF000310650913206213079F56417750760F577
:102F0000E0913E06F0913F0620912B0630912C0671
:102F1000E617F707C0F42F5F3F4F8217930728F09B
:102F200030932C0620932B0604C090932C0680939C
:102F30002B0620912B0630912C062536310560F0AA
:102F400024E630E005C02115310531F0215031096A
:102F500030932C0620932B064617570708F088C09D
:102F600020914606211133C020913E0630913F0644
:102F700024173507D0F460912B0670912C066F5FF3
:102F80007F4F6536710510F064E670E070932C0693
:102F900060932B0660912B0670912C06861797077D
:102FA00020F490932C0680932B064217530708F0C9
:102FB0005FC080912B0690912C06009729F0019715
:102FC00090932C0680932B06241B350B38C02130A0
:102FD00009F04EC020910B0630910C066091190645
:102FE00070911A0626173707D0F440912B0650919E
:102FF0002C064F5F5F4F4536510510F044E650E018
:1030000050932C0640932B0640912B0650912C0692
:103010008417950720F490932C0680932B06621753
:10302000730730F580912B0690912C06009729F0BC
:10303000019790932C0680932B06261B370B2B3081
:103040003105B0F080912B0690912C060A9720F460
:1030500010922C0610922B0680912B0690912C0634
:103060008A30910528F00A9790932C0680932B06BE
:10307000CF9108954091E5055091E60520911B06FA
:1030800030911C06429FC001439F900D529F900DAE
:1030900011246AE070E00E94DD3F70934206609365
:1030A000410680912B0690912C068536910530F0D3
:1030B00084E690E090932C0680932B06809129065D
:1030C00090E020912B0630912C068217930720F474
:1030D00090932C0680932B0620912D0640913E065E
:1030E00050913F06211110C04639510538F424E6AD
:1030F00030E030932C0620932B0606C0463951054C
:1031000019F021E020932D0620912D06E091310643
:10311000F0913206213059F56E177F0740F5209166
:103120002B0630912C0646175707C0F42F5F3F4FF0
:103130008217930728F030932C0620932B0604C0A7
:1031400090932C0680932B0620912B0630912C0611
:103150002536310560F024E630E005C02115310543
:1031600031F02150310930932C0620932B06E617BD
:10317000F70708F046C04E175F07D0F420912B06E2
:1031800030912C062F5F3F4F2536310510F024E695
:1031900030E030932C0620932B0620912B063091A3
:1031A0002C068217930720F490932C0680932B060D
:1031B000E417F50730F580912B0690912C060097C7
:1031C00029F0019790932C0680932B06CA018E1B41
:1031D0009F0B0B97B0F080912B0690912C060A97CD
:1031E00020F410922C0610922B0680912B069091C1
:1031F0002C068A30910528F00A9790932C0680932C
:103200002B0680912A0690E020917D0630917E0663
:103210008217930720F490937E0680937D06E4172F
:10322000F50770F480917D0690917E0601968536B3
:10323000910510F084E690E090937E0680937D06E1
:1032400008954091E5055091E60520911B063091C7
:103250001C06429FC001439F900D529F900D112468
:103260006AE070E00E94DD3F709342066093410681
:1032700080912B0690912C068536910530F084E6DE
:1032800090E090932C0680932B068091290690E085
:1032900020912B0630912C068217930720F49093EF
:1032A0002C0680932B0620912D06211114C020910D
:1032B0003E0630913F062639310538F424E630E0E9
:1032C00030932C0620932B0606C02639310519F0C1
:1032D00021E020932D0620912D064091310650913A
:1032E0003206213079F56417750760F5E0913E06E6
:1032F000F0913F0620912B0630912C06E617F70738
:10330000C0F42F5F3F4F8217930728F030932C06AD
:1033100020932B0604C090932C0680932B062091BB
:103320002B0630912C062536310560F024E630E07E
:1033300005C02115310531F02150310930932C069B
:1033400020932B064617570708F04AC020913E06E7
:1033500030913F0624173507D0F460912B06709109
:103360002C066F5F7F4F6536710510F064E670E0E4
:1033700070932C0660932B0660912B0670912C069F
:103380008617970720F490932C0680932B064217FC
:10339000530730F580912B0690912C06009729F069
:1033A000019790932C0680932B06241B350B2B3012
:1033B0003105B0F080912B0690912C060A9720F4ED
:1033C00010922C0610922B0680912B0690912C06C1
:1033D0008A30910528F00A9790932C0680932B064B
:1033E0000895BC9A80917D06880F81BF139A8091C1
:1033F0002B06880F80938600809114069091150605
:10340000892B11F4A5D9C6DA80911406909115067E
:10341000019729F410922C0610922B06EFDB809175
:10342000140690911506029729F410927E061092C8
:103430007D06F2DC8091140690911506049709F43C
:1034400019DE8091140690911506059709F412DE95
:103450008091140690911506069709F4F2CE08950E
:1034600063EC70E084E992E00E942F4362EC71E02B
:1034700086E992E00E942F4366E170E088E992E0DD
:103480000E942F4366E170E08AE992E00E942F4398
:1034900061E070E08CE992E00E942F43A8956EE60F
:1034A00070E08EE992E00E942F4364E670E080EACB
:1034B00092E00E942F4364E670E082EA92E00E946C
:1034C0002F4360E070E084EA92E00E942F43A895C9
:1034D00060E070E086EA92E00E942F4360E070E0D6
:1034E00088EA92E00E942F4360E070E08AEA92E06E
:1034F0000E942F4360E070E08CEA92E00E942F432C
:1035000060E070E08EEA92E00E942F4360E070E09D
:1035100080EB92E00E942F43A89566EE70E086E76C
:1035200092E00E942F4362EC71E088E792E00E94F3
:103530002F4366E170E08AE792E00E942F4366E144
:1035400070E08CE792E00E942F4361E070E08EE72C
:1035500092E00E942F43A89563E770E080E892E034
:103560000E942F4364E670E082E892E00E942F43BD
:1035700064E670E084E892E00E942F4360E070E02F
:1035800086E892E00E942F4360E070E088E892E0D5
:103590000E942F4360E070E08AE892E00E942F438F
:1035A000A89560E070E08CE892E00E942F4360E014
:1035B00070E08EE892E00E942F4360E070E080E9C6
:1035C00092E00E942F4360E070E082E992E00E9466
:1035D0002F43A89566EE70E088E592E00E942F43A5
:1035E00062EC71E08AE592E00E942F4366E170E0B0
:1035F0008CE592E00E942F4366E170E08EE592E058
:103600000E942F4361E070E080E692E00E942F4329
:10361000A89563E770E082E692E00E942F4364E69B
:1036200070E084E692E00E942F4364E670E086E654
:1036300092E00E942F4360E070E088E692E00E94F2
:103640002F4360E070E08AE692E00E942F4360E042
:1036500070E08CE692E00E942F43A89560E070E055
:103660008EE692E00E942F4360E070E080E792E0F7
:103670000E942F4360E070E082E792E00E942F43B7
:1036800060E070E084E792E00E942F43A89566E92D
:1036900070E08AE392E00E942F4368EC70E08CE3D4
:1036A00092E00E942F4366E170E08EE392E00E9478
:1036B0002F4366E170E080E492E00E942F4361E0D6
:1036C00070E082E492E00E942F43A89563E770E0E7
:1036D00084E492E00E942F4364E670E086E492E086
:1036E0000E942F4364E670E088E492E00E942F433A
:1036F00060E070E08AE492E00E942F4360E070E0B6
:103700008CE492E00E942F4360E070E08EE492E04F
:103710000E942F43A89560E070E080E592E00E944F
:103720002F4360E070E082E592E00E942F4360E06A
:1037300070E084E592E00E942F4360E070E086E54F
:1037400092E00E942F43A8956EEB70E08CE192E02E
:103750000E942F4368EC70E08EE192E00E942F43BC
:1037600066E170E080E292E00E942F4366E170E043
:1037700082E292E00E942F4361E070E084E292E0F6
:103780000E942F43A89564E670E086E292E00E94D2
:103790002F4364E670E088E292E00E942F4364E6E3
:1037A00070E08AE292E00E942F4360E070E08CE2D9
:1037B00092E00E942F4360E070E08EE292E00E946F
:1037C0002F4360E070E080E392E00E942F43A895D1
:1037D00060E070E082E392E00E942F4360E070E0DE
:1037E00084E392E00E942F4360E070E086E392E081
:1037F0000E942F4360E070E088E392E00E942F4334
:10380000A89566EE70E08EEF91E00E942F4362EC87
:1038100071E080E092E00E942F4366E170E082E078
:1038200092E00E942F4366E170E084E092E00E9403
:103830002F4361E070E086E092E00E942F43A8955C
:1038400063E770E088E092E00E942F4364E670E056
:103850008AE092E00E942F4364E670E08CE092E000
:103860000E942F4360E070E08EE092E00E942F43C0
:1038700060E070E080E192E00E942F4360E070E041
:1038800082E192E00E942F43A89560E070E084E11D
:1038900092E00E942F4360E070E086E192E00E9497
:1038A0002F4360E070E088E192E00E942F4360E0E7
:1038B00070E08AE192E00E942F43A89566EE70E0E6
:1038C00080EE91E00E942F4362EC71E082EE91E085
:1038D0000E942F4366E170E084EE91E00E942F4346
:1038E00066E170E086EE91E00E942F4361E070E0B7
:1038F00088EE91E00E942F43A89563E770E08AEE7E
:1039000091E00E942F4364E670E08CEE91E00E940B
:103910002F4364E670E08EEE91E00E942F4360E05A
:1039200070E080EF91E00E942F4360E070E082EF52
:1039300091E00E942F4360E070E084EF91E00E94EC
:103940002F43A89560E070E086EF91E00E942F433E
:1039500060E070E088EF91E00E942F4360E070E04B
:103960008AEF91E00E942F4360E070E08CEF91E0DD
:103970000E942F43A89563EC70E084EA91E00E94D6
:103980002F4366E170E088EA91E00E942F4361E0F6
:1039900070E08CEA91E00E942F436FE070E08EEAC5
:1039A00091E00E942F43A89564E670E080EB91E0DF
:1039B0000E942F4361E070E08AEB91E00E942F4368
:1039C00063EC70E08CEB91E00E942F436AE070E0C2
:1039D0008EEB91E00E942F43A89562EC71E08CE49D
:1039E00091E00E942F4366E170E080E591E00E9443
:1039F0002F4361E070E082E591E00E942F436EE684
:103A000070E084E591E00E942F43A89564E670E0A1
:103A100088E591E00E942F4362E070E080E691E04B
:103A20000E942F4362EC71E082EF90E00E942F43EE
:103A300066E170E084EF90E00E942F4362E170E065
:103A400086EF90E00E942F43A89564E670E08CEF2B
:103A500090E00E942F4364E670E08EEF90E00E94B9
:103A60002F4364E070E086E091E00E942F436CE217
:103A700071E08CE091E00E942F43A89562EC71E028
:103A800088E990E00E942F4366E170E08AE990E0C7
:103A90000E942F4366E170E08CE990E00E942F4382
:103AA00061E070E08EE990E00E942F43A8956EE6F9
:103AB00070E080EA90E00E942F4364E670E082EAC2
:103AC00090E00E942F4364E670E084EA90E00E9458
:103AD0002F4365E070E08CEA90E00E942F43A895A8
:103AE00062EC71E08EE390E00E942F4366E170E0AB
:103AF00082E490E00E942F4361E070E084E490E073
:103B00000E942F436EE670E086E490E00E942F430F
:103B1000A89564E670E08AE490E00E942F4366E096
:103B200070E082E590E00E942F4363EC70E084E94E
:103B300092E00E942F43A89508956FE070E088EB13
:103B400092E00E942F436FE070E086EB92E00E94CB
:103B50002F436FE070E084EB92E00E942F4361E01E
:103B600083EB92E00E94224361E082EB92E00C94AE
:103B700022438FB9779BFECF8FB10895CF93A39A3D
:103B8000AB9AAB9880E0F5DFC82F80E0F2DFAB9A0C
:103B90006C2F70E0762F6627682B687F7F7723E095
:103BA000769567952A95E1F780E090E00E94EC3EDB
:103BB00020E030E040E85EE30E94523F0E94C03EB9
:103BC00070930C0660930B06CB01CF910895CF93B1
:103BD000A79AAF9AAF9880E0CCDFC82F80E0C9DF0A
:103BE000AF9A6C2F70E0762F6627682B687F7F77FF
:103BF00023E0769567952A95E1F780E090E00E94B2
:103C0000EC3E20E030E040E85EE30E94523F0E943C
:103C1000C03E70933F0660933E06CB01CF9108955E
:103C200080E091E0909383068093820680910C0659
:103C30008F9380910B068F938EE091E09F938F93EB
:103C40000E942C408DE08A95F1F700008091E605F6
:103C50008F938091E5058F9388E191E09F938F93F7
:103C60000E942C409DE09A95F1F7000080912C066F
:103C70008F9380912B068F9382E291E09F938F9395
:103C80000E942C408DE08A95F1F7000080917E061D
:103C90008F9380917D068F938DE291E09F938F9318
:103CA0000E942C409DE09A95F1F7000087E391E097
:103CB0009F938F930E942C408DE08A95F1F700002E
:103CC00080913F068F9380913E068F938FE391E022
:103CD0009F938F930E942C40A8958DB79EB74696D0
:103CE0000FB6F8949EBF0FBE8DBF809112069091C3
:103CF0001306892B41F488E491E09F938F930E94EF
:103D00002C400F900F90A895809112069091130669
:103D1000019741F48FE491E09F938F930E942C4090
:103D20000F900F909DE09A95F1F70000E091140636
:103D3000F0911506E830F10508F09CC0E25AFF4FFB
:103D40000C94F13F86E591E09F938F930E942C4065
:103D5000A8950F900F90E09171068E2F90E088301B
:103D6000910508F087C0FC01EA59FF4F0C94F13F20
:103D700085E691E071C085E791E06EC08DEA91E043
:103D80006BC08CEB91E068C08BEC91E065C08AED74
:103D900091E09F938F930E942C40A8950F900F90D5
:103DA00080911D06813009F452C008F44DC0823064
:103DB00009F450C008958AEE91E09F938F930E947A
:103DC0002C40A8950F900F9080912406813009F423
:103DD0003EC0D0F1823009F43DC008958BEF91E0F0
:103DE00042C089E092E09F938F930E942C40A89557
:103DF0000F900F9080917C06813049F128F182303C
:103E000049F108958AE192E09F938F930E942C409C
:103E1000A8950F900F90809170068130C1F0A0F0AE
:103E20008230C1F008958DE292E09F938F930E94BB
:103E30002C40A8950F900F9080916D06813039F03D
:103E400018F0823039F0089580E891E005C08FE8DD
:103E500091E002C08EE991E09F938F930E942C40E5
:103E600007C08FE392E09F938F930E942C40A89508
:103E70000F900F900895CF92DF92EF92FF920F93E1
:103E80001F93CF93DF9300D000D0CDB7DEB78091E2
:103E9000120690911306019709F028C1809125061A
:103EA00090912606892BD9F40FE110E024E230E04E
:103EB0004AE550E064E670E088E090E00E94A404E7
:103EC00024E230E04AE550E064E670E08FED90E0F7
:103ED0000E94A404A895A49AAC980E94EB07CC2455
:103EE000C394D12C8091120690911306019709F08A
:103EF000FDC0A89595DE80917306909174068A3571
:103F0000910549F42FEF8DE399E4215080409040D2
:103F1000E1F700C00000A89503E02FE130E04FEF8B
:103F20005FEF69E170E085E890E00E940411809104
:103F30006300A8951C821B821A821982BE016F5FE2
:103F40007F4FCE0103960E94543E8B819C81843129
:103F5000954088F489819A81883D9E4060F48981EA
:103F60009A81853C994038F0D0922606C092250669
:103F70001092350609D48B819C818431954008F0DC
:103F80003FC089819A818C3D9540D0F589819A8185
:103F9000853F9140A8F1D0922606C0922506109246
:103FA00047068091140690911506892B11F40E9402
:103FB000B3308091140690911506019711F40E9478
:103FC0004F398091140690911506029711F40E94C2
:103FD000563A8091140690911506049711F40E94A8
:103FE0005B3B8091140690911506059709F454D512
:103FF0008091140690911506069711F40E94AB2F3C
:104000008B819C81853C994098F089819A818C3D77
:10401000954070F489819A81853F914048F01092D3
:104020002606109225068FE190E00E94190623DFF4
:10403000A5DD0E94D20EA8958FEF91EE24E081506D
:1040400090402040E1F700C00000C1DDA8950E942B
:10405000580FE0902B06F0902C0603E02FE130E0A3
:104060004FEF5FEF6EE670E08CE190E00E94DF05BD
:10407000E0907D06F0907E062FE130E04FEF5FEF9D
:104080006EE670E080EF90E00E94DF050E94CF10A6
:104090008091120690911306892B09F023CFA895E1
:1040A0000E941912A8950E948B110E94EB070FE144
:1040B00010E024E230E04AE550E064E670E088E099
:1040C00090E00E94A40424E230E04AE550E064E677
:1040D00070E08FED90E00E94A4041092E60510922B
:1040E000E5051092260610922506FCCE0F900F9043
:1040F0000F900F90DF91CF911F910F91FF90EF9054
:10410000DF90CF900895EF92FF920F931F93CF937C
:1041100080913406813009F04BC18FE190E00E941C
:1041200019060E94C10B85E080933A06C5E0809194
:104130003406813009F03CC10E94DD0C80913A06C2
:104140008230D9F4809166068F5F809366060FE116
:1041500010E02CE330E046EE50E069E670E081E0EC
:1041600090E00E94A40422E330E043EC50E068E2D7
:1041700070E088E090E00E94A40480913A068330C9
:10418000D9F4809166068150809366060FE110E0B5
:104190002CE330E046EE50E069E670E081E090E02C
:1041A0000E94A40422E330E043EC50E068E270E0B7
:1041B00088E090E00E94A40480916606853010F0AB
:1041C0001092660680916606823081F1B8F48823E9
:1041D000D9F0813009F0C1C076E8E72E75E0F72EFE
:1041E00001E02FE130E04FEF5FEF6CE370E088E03B
:1041F00090E00E94990586EB92E029C08330B1F1EE
:10420000843009F471C0A9C0EFE9EE2EE5E0FE2E7E
:1042100001E02FE130E04FEF5FEF6CE370E08FE003
:1042200090E00E94990588EB92E011C06AE7E62EC3
:1042300065E0F62E01E02FE130E04FEF5FEF6CE339
:1042400070E082E390E00E94990584EB92E00E9486
:1042500014437C0103E02FE130E04FEF5FEF62E8B1
:1042600070E080E590E00E94DF0577C042E6E42E32
:1042700045E0F42E01E02FE130E04FEF5FEF6CE31B
:1042800070E088E290E00E94990550E7E52E55E045
:10429000F52E02E02FE130E04FEF5FEF62E870E0D3
:1042A00088E290E00E94990580913A06811119C038
:1042B000D7D843DC3CE2E32E35E0F32E2FE130E0AB
:1042C0004FEF5FEF62E870E088E290E00E949905AE
:1042D0002FEF89E698E1215080409040E1F700C03F
:1042E0000000C0933A0639C021E5E22E25E0F22E07
:1042F00001E02FE130E04FEF5FEF6CE370E08EE123
:1043000090E00E94990583EB92E00E940C4381307B
:1043100079F493E4E92E95E0F92E03E02FE130E003
:104320004FEF5FEF62E870E080E590E00E94990552
:1043300083EB92E00E940C4381110FC08EE3E82EC4
:1043400085E0F82E03E02FE130E04FEF5FEF62E809
:1043500070E080E590E00E94990580913A068130F6
:1043600089F41092340610922606109225068FE1E9
:1043700090E00E94190681E090E0909313068093EC
:10438000120679DD80913A06811106C081E08093A2
:1043900034061092780612D0C0933A062FE785EBC8
:1043A00091E0215080409040E1F700C00000BFCE76
:1043B000CF911F910F91FF90EF900895BF92CF92F0
:1043C000DF92EF92FF920F931F93CF93DF93809131
:1043D00078068111CFC185E080933A06C9E1D0E02B
:1043E00025E0C22ED12C35E0B32E809178068111C4
:1043F000C1C180916606813009F46FC038F0823007
:1044000009F4DDC0843009F441C1A4C188EB92E015
:104410000E9414437C0103E02FE130E040E058EFBC
:1044200062E870E080E590E00E94DF0588EB92E0B2
:104430000E94144390933906809338060E94DD0C45
:1044400080913A068230A9F480913806909139061D
:10445000019690933906809338060FE110E02CE323
:1044600030E046EE50E069E670E081E090E00E94C6
:10447000A40480913A068330A9F480913806909183
:104480003906019790933906809338060FE110E0C2
:104490002CE330E046EE50E069E670E081E090E029
:1044A0000E94A40480913806909139064A9720F022
:1044B000D0933906C093380680913806909139061A
:1044C0000A9720F4D0933906C093380660913806D5
:1044D0007091390688EB92E066C086EB92E00E940C
:1044E00014437C0103E02FE130E040E058EF62E844
:1044F00070E080E590E00E94DF0586EB92E00E948C
:10450000144390931806809317060E94DD0C809147
:104510003A068230A9F48091170690911806019608
:1045200090931806809317060FE110E02CE330E01B
:1045300046EE50E069E670E081E090E00E94A4045D
:1045400080913A068330A9F480911706909118065D
:10455000019790931806809317060FE110E02CE363
:1045600030E046EE50E069E670E081E090E00E94C5
:10457000A40480911706909118064A9720F0D093D2
:104580001806C093170680911706909118060A978F
:1045900020F4D0931806C093170660911706709107
:1045A000180686EB92E00E942F432FE788E391E004
:1045B000215080409040E1F700C00000CBC084EB68
:1045C00092E00E9414437C0103E02FE130E040E0E0
:1045D00058EF62E870E080E590E00E94DF0584EB30
:1045E00092E00E94144390933706809336060E940F
:1045F000DD0C80913A068230A9F4809136069091C4
:104600003706019690933706809336060FE110E047
:104610002CE330E046EE50E069E670E081E090E0A7
:104620000E94A40480913A068330A9F48091360652
:1046300090913706019790933706809336060FE1E5
:1046400010E02CE330E046EE50E069E670E081E0F7
:1046500090E00E94A40480913606909137064F970F
:1046600020F0D0923706C09236068091360690919F
:104670003706059720F4D0923706C092360660912F
:1046800036067091370684EB92E08DCF83EB92E093
:104690000E940C438093DB050E94DD0C80913A065A
:1046A000823089F48091DB058F5F8093DB050FE119
:1046B00010E02CE330E046EE50E069E670E081E087
:1046C00090E00E94A40480913A06833089F480919E
:1046D000DB0581508093DB050FE110E02CE330E037
:1046E00046EE50E069E670E081E090E00E94A404AC
:1046F0008091DB05823010F01092DB058091DB05A4
:10470000813079F493E4E92E95E0F92E03E02FE16E
:1047100030E040E058EF62E870E080E590E00E9411
:1047200099058091DB0581110FC08EE3E82E85E0AD
:10473000F82E03E02FE130E040E058EF62E870E04F
:1047400080E590E00E9499056091DB0583EB92E0A3
:104750000E94224380913A06813049F48093780682
:10476000809334068FE190E00E941906CCDCB09271
:104770003A063BCEDF91CF911F910F91FF90EF90C2
:10478000DF90CF90BF9008954F925F926F927F928B
:104790008F929F92AF92BF92CF92DF92EF92FF9251
:1047A0000F931F93CF93DF9380913506811163C1DF
:1047B0008FE190E00E9419060E94330B85E0809300
:1047C0003A061092340610922E0655245394C7E0F0
:1047D000D0E0A6E0CA2ED12CB5E0AB2EB12C14E06F
:1047E000812E912C03E0602E712C85E0482E809163
:1047F0003506811140C10E94DD0C80913A0682305D
:1048000089F480912E068F5F80932E060FE110E0D1
:104810002CE330E046EE50E069E670E081E090E0A5
:104820000E94A40480913A06833089F480912E0678
:10483000815080932E060FE110E02CE330E046EE2D
:1048400050E069E670E081E090E00E94A40480916D
:104850002E06893010F010922E06E0912E068E2F33
:1048600090E08930910508F0D4C0FC01E259FF4F77
:104870000C94F13FFEE0EF2EF5E0FF2E02E02FE179
:1048800030E04FEF5FEF62E870E088E090E00E9478
:104890009905109234061092150610921406B9C0AC
:1048A000E0E0EE2EE5E0FE2E02E02FE130E04FEFFB
:1048B0005FEF68E770E088E090E00E949905109251
:1048C000340681E090E013C072EFE72E74E0F72E1B
:1048D00002E02FE130E04FEF5FEF68E770E088E043
:1048E00090E00E9499051092340682E090E0909347
:1048F0001506809314068DC066EEE62E64E0F62E53
:1049000002E02FE130E04FEF5FEF68E770E088E012
:1049100090E00E94990510923406709215066092FC
:10492000140677C054EDE52E54E0F52E02E02FE199
:1049300030E04FEF5FEF68E770E088E090E00E94C2
:10494000990510923406909215068092140661C063
:104950003EECE32E34E0F32E02E02FE130E04FEFA7
:104960005FEF6EE670E088E290E00E94990544EC0B
:10497000E42E44E0F42E2FE130E04FEF5FEF67E8E4
:1049800070E08FE090E00E94990510923406B0929A
:104990001506A09214063DC027EBE22E24E0F22E6D
:1049A00002E02FE130E04FEF5FEF68E770E088E072
:1049B00090E00E94990510923406D0921506C0929C
:1049C000140627C099E9E92E94E0F92E02E02FE1C0
:1049D00030E04FEF5FEF68E770E088E090E00E9422
:1049E000990510923406D0931506C093140611C091
:1049F00083EAE82E84E0F82E02E02FE130E04FEF6A
:104A00005FEF68E770E082E090E00E9499055092C5
:104A1000340680913A06813011F580913406813058
:104A200059F41092150610921406109235068FE173
:104A300090E00E94190667DB509235061092260618
:104A40001092250680911406909115069093020607
:104A5000809301068FE190E00E9419060CDA4092E3
:104A60003A062FEF80E792E0215080409040E1F736
:104A700000C00000BCCEDF91CF911F910F91FF903D
:104A8000EF90DF90CF90BF90AF909F908F907F90EE
:104A90006F905F904F900895EF92FF920F931F9346
:104AA000CF93DF93A895809147068111F4C08FE1E1
:104AB00090E00E9419060E944F0C8091700690E0D1
:104AC0009093200680931F0685E080933A06C1E00C
:104AD000D5E0809147068111DEC0A8950E94DD0CCB
:104AE00080913A068230A9F480911F0690912006A9
:104AF00001969093200680931F060FE110E02CE3AF
:104B000030E046EE50E069E670E081E090E00E941F
:104B1000A40480913A068330A9F480911F069091F5
:104B2000200601979093200680931F060FE110E066
:104B30002CE330E046EE50E069E670E081E090E082
:104B40000E94A40480911F0690912006039720F0F4
:104B50001092200610921F0680911F069091200649
:104B60008130910589F1D0F0029709F046C081E7C4
:104B7000E82E84E0F82E02E02FE130E04FEF5FEF07
:104B80006DE770E088E290E00E94990582E08093F2
:104B900070064EE150E06AE570E02BC025E8E22E99
:104BA00024E0F22E02E02FE130E04FEF5FEF6DE7FF
:104BB00070E088E290E00E949905109270064EE144
:104BC00050E066E970E015C09BE7E92E94E0F92E0D
:104BD00002E02FE130E04FEF5FEF6DE770E088E239
:104BE00090E00E949905C09370064EE150E068E79E
:104BF00070E08BEE95E00E94FC4280913A068111B4
:104C00000FC0A895C093470610922606109225065D
:104C1000C09335068FE190E00E941906A8952BD924
:104C200080913A06813059F5A895809347061092F5
:104C3000260610922506809335068FE190E00E94AB
:104C40001906A89510927F0680917006813069F050
:104C500038F0823091F44EE150E06AE570E009C02E
:104C60004EE150E066E970E004C04EE150E068E7D4
:104C700070E08BEE95E00E94FC42A89513D0D09393
:104C80003A062FEF80E792E0215080409040E1F714
:104C900000C000001ECFDF91CF911F910F91FF90B8
:104CA000EF900895EF92FF920F931F93CF9380910F
:104CB0007F0681110C94A52F8FE190E00E941906C8
:104CC0000E94450D85E080933A06C5E080917F06FD
:104CD00081110C94A52F0E94DD0C80913A06823040
:104CE000D9F480916B068F5F80936B060FE110E023
:104CF0002CE330E046EE50E069E670E081E090E0C1
:104D00000E94A40422E330E043EC50E068E270E04B
:104D100088E090E00E94A40480913A068330D9F4A0
:104D200080916B06815080936B060FE110E02CE3BD
:104D300030E046EE50E069E670E081E090E00E94ED
:104D4000A40422E330E043EC50E068E270E088E045
:104D500090E00E94A40480916B068E3010F01092B7
:104D60006B06E0916B068E2F90E08E30910508F077
:104D700097C7FC01E958FF4F8091140690911506E2
:104D80000C94F13F892B61F57BE2E72E74E0F72E5E
:104D900001E02FE130E04FEF5FEF62E370E08FE082
:104DA00090E00E949905E4E2EE2EE4E0FE2E2FE171
:104DB00030E04FEF5FEF66E470E08CE390E00E943C
:104DC0009905E090EB05F090EC0503E02FE130E071
:104DD0004FEF5FEF62E870E080E590E00E94DF0552
:104DE0008091140690911506019709F07BC65BE24D
:104DF000E52E54E0F52E01E02FE130E04FEF5FEFBC
:104E000062E370E08FE090E00E94990564E2E62E94
:104E100064E0F62E2FE130E04FEF5FEF66E470E0E4
:104E20008CE390E00E949905E090EB05F090EC0592
:104E30004EC6892B61F53CE0E32E34E0F32E01E011
:104E40002FE130E04FEF5FEF62E370E08FE090E042
:104E50000E9499054EEFE42E43E0F42E2FE130E05E
:104E60004FEF5FEF66E470E08CE390E00E949905FD
:104E7000E090ED05F090EE0503E02FE130E04FEF1C
:104E80005FEF62E870E080E590E00E94DF058091CE
:104E90001406909115068130910531F480916B06CE
:104EA0008F5F80936B062EC0029761F59CE0E92E20
:104EB00094E0F92E01E02FE130E04FEF5FEF62E385
:104EC00070E08FE090E00E9499052EEFE22E23E043
:104ED000F22E2FE130E04FEF5FEF66E470E08CE3FD
:104EE00090E00E949905E090ED05F090EE0503E05A
:104EF0002FE130E04FEF5FEF62E870E080E590E097
:104F00000E94DF058091140690911506049761F5C3
:104F10000CE0E02E04E0F02E01E02FE130E04FEF56
:104F20005FEF62E370E08FE090E00E9499058EEF02
:104F3000E82E83E0F82E2FE130E04FEF5FEF66E4DC
:104F400070E08CE390E00E949905E090ED05F09010
:104F5000EE0503E02FE130E04FEF5FEF62E870E035
:104F600080E590E00E94DF0580911406909115067F
:104F7000059761F5BCE0EB2EB4E0FB2E01E02FE1DC
:104F800030E04FEF5FEF62E370E08FE090E00E946F
:104F900099051EEFE12E13E0F12E2FE130E04FEFE7
:104FA0005FEF66E470E08CE390E00E949905E0908A
:104FB000ED05F090EE0503E02FE130E04FEF5FEFFD
:104FC00062E870E080E590E00E94DF0580911406C1
:104FD00090911506069709F063C6FCE0EF2EF4E009
:104FE000FF2E01E02FE130E04FEF5FEF62E370E072
:104FF0008FE090E00E949905AEEFEA2EA3E0FA2E32
:105000002FE130E04FEF5FEF66E470E08CE390E07B
:105010000E949905E090ED05F090EE05D8C4892B2B
:1050200061F576EEE72E73E0F72E01E02FE130E038
:105030004FEF5FEF62E370E08FE090E00E94990530
:10504000EEECEE2EE3E0FE2E2FE130E04FEF5FEFCF
:1050500066E470E08FE090E00E949905E090EF0533
:10506000F090F00503E02FE130E04FEF5FEF62E8F2
:1050700070E080E590E00E94DF0580911406909139
:105080001506019709F02EC556EEE52E53E0F52ED4
:1050900001E02FE130E04FEF5FEF62E370E08FE07F
:1050A00090E00E9499056EECE62E63E0F62E2FE16B
:1050B00030E04FEF5FEF66E470E08FE090E00E9439
:1050C0009905E090EF05F090F00501C5892B61F599
:1050D00036EBE32E33E0F32E01E02FE130E04FEF2B
:1050E0005FEF62E370E08FE090E00E9499054EE987
:1050F000E42E43E0F42E2FE130E04FEF5FEF66E463
:1051000070E08FE090E00E949905E090F105F0904A
:10511000F20503E02FE130E04FEF5FEF62E870E06F
:1051200080E590E00E94DF058091140690911506BD
:105130008130910531F480916B068F5F80936B060F
:105140002EC0029761F596EBE92E93E0F92E01E06F
:105150002FE130E04FEF5FEF62E370E08FE090E02F
:105160000E9499052EE9E22E23E0F22E2FE130E095
:105170004FEF5FEF66E470E08FE090E00E949905EA
:10518000E090F105F090F20503E02FE130E04FEF01
:105190005FEF62E870E080E590E00E94DF058091BB
:1051A000140690911506049761F506EBE02E03E0D6
:1051B000F02E01E02FE130E04FEF5FEF62E370E0AF
:1051C0008FE090E00E9499058EE9E82E83E0F82EAA
:1051D0002FE130E04FEF5FEF66E470E08FE090E0AA
:1051E0000E949905E090F105F090F20503E02FE1AF
:1051F00030E04FEF5FEF62E870E080E590E00E9402
:10520000DF058091140690911506059761F5B6EBC0
:10521000EB2EB3E0FB2E01E02FE130E04FEF5FEF2C
:1052200062E370E08FE090E00E9499051EE9E12EB4
:1052300013E0F12E2FE130E04FEF5FEF66E470E016
:105240008FE090E00E949905E090F105F090F20562
:1052500003E02FE130E04FEF5FEF62E870E080E5C0
:1052600090E00E94DF058091140690911506069744
:1052700009F016C5F6EBEF2EF3E0FF2E01E02FE16B
:1052800030E04FEF5FEF62E370E08FE090E00E946C
:105290009905AEE9EA2EA3E0FA2E2FE130E04FEFB8
:1052A0005FEF66E470E08FE090E00E949905E09087
:1052B000F105F090F2058BC3892BC9F5E6E8EE2ED7
:1052C000E3E0FE2E01E02FE130E04FEF5FEF6CE313
:1052D00070E08FE090E00E9499058091F305909135
:1052E000F405019779F473E4E72E75E0F72E03E0F7
:1052F0002FE130E04FEF5FEF62E870E080E590E093
:105300000E9499058091F3059091F405892B79F419
:105310006EE3E62E65E0F62E03E02FE130E04FEF7E
:105320005FEF62E870E080E590E00E94990580916F
:105330001406909115060197C9F556E8E52E53E03D
:10534000F52E01E02FE130E04FEF5FEF6CE370E00E
:105350008FE090E00E9499058091F3059091F4050B
:10536000019779F443E4E42E45E0F42E03E02FE1C5
:1053700030E04FEF5FEF62E870E080E590E00E9480
:1053800099058091F3059091F405892B79F43EE31A
:10539000E32E35E0F32E03E02FE130E04FEF5FEF37
:1053A00062E870E080E590E00E9499058091140623
:1053B000909115060297C9F526E8E22E23E0F22E19
:1053C00001E02FE130E04FEF5FEF6CE370E08FE042
:1053D00090E00E9499058091F3059091F405019762
:1053E00079F493E4E92E95E0F92E03E02FE130E023
:1053F0004FEF5FEF62E870E080E590E00E94990572
:105400008091F3059091F405892B79F48EE3E82ED1
:1054100085E0F82E03E02FE130E04FEF5FEF62E828
:1054200070E080E590E00E949905809114069091CB
:1054300015069C01245031092230310508F4F6C3C9
:10544000069709F02DC406E8E02E03E0F02E01E0F7
:105450002FE130E04FEF5FEF6CE370E08FE090E022
:105460000E9499058091F3059091F405019779F4D4
:1054700013E4E12E15E0F12E03E02FE130E04FEFD1
:105480005FEF62E870E080E590E00E94990580910E
:10549000F3059091F405892B09F002C4BEE3EB2ECD
:1054A000B5E0FB2E03E02FE130E04FEF5FEF62E865
:1054B00070E080E590E00E949905F2C3892B61F5C8
:1054C000FEE6EF2EF3E0FF2E01E02FE130E04FEF9C
:1054D0005FEF62E370E08FE090E00E949905A6E53F
:1054E000EA2EA3E0FA2E2FE130E04FEF5FEF66E403
:1054F00070E08FE090E00E949905E090F505F09053
:10550000F60503E02FE130E04FEF5FEF62E870E077
:1055100080E590E00E94DF058091140690911506C9
:10552000019761F57EE6E72E73E0F72E01E02FE1AB
:1055300030E04FEF5FEF62E370E08FE090E00E94B9
:105540009905E6E5EE2EE3E0FE2E2FE130E04FEF89
:105550005FEF66E470E08FE090E00E949905E090D4
:10556000F505F090F60503E02FE130E04FEF5FEF37
:1055700062E870E080E590E00E94DF05809114060B
:1055800090911506029761F55EE6E52E53E0F52E43
:1055900001E02FE130E04FEF5FEF62E370E08FE07A
:1055A00090E00E94990566E5E62E63E0F62E2FE175
:1055B00030E04FEF5FEF66E470E08FE090E00E9434
:1055C0009905E090F505F090F60503E02FE130E055
:1055D0004FEF5FEF62E870E080E590E00E94DF054A
:1055E00080911406909115069C01245031092230B7
:1055F000310508F41BC3069709F052C33EE6E32EBB
:1056000033E0F32E01E02FE130E04FEF5FEF62E394
:1056100070E08FE090E00E94990546E5E42E43E0BB
:10562000F42E2FE130E04FEF5FEF66E470E08FE0A3
:1056300090E00E949905E090F505F090F605C7C14D
:10564000892B61F59EE3E92E93E0F92E01E02FE12D
:1056500030E04FEF5FEF62E370E08FE090E00E9498
:10566000990526E2E22E23E0F22E2FE130E04FEF03
:105670005FEF66E470E08FE090E00E949905E090B3
:10568000F705F090F80503E02FE130E04FEF5FEF12
:1056900062E870E080E590E00E94DF0580911406EA
:1056A00090911506019761F50EE3E02E03E0F02ED0
:1056B00001E02FE130E04FEF5FEF62E370E08FE059
:1056C00090E00E94990586E2E82E83E0F82E2FE113
:1056D00030E04FEF5FEF66E470E08FE090E00E9413
:1056E0009905E090F705F090F80503E02FE130E030
:1056F0004FEF5FEF62E870E080E590E00E94DF0529
:1057000080911406909115068230910531F48091B4
:105710006B068F5F80936B062EC0049761F5BEE326
:10572000EB2EB3E0FB2E01E02FE130E04FEF5FEF17
:1057300062E370E08FE090E00E94990516E2E12EAE
:1057400013E0F12E2FE130E04FEF5FEF66E470E001
:105750008FE090E00E949905E090F705F090F80541
:1057600003E02FE130E04FEF5FEF62E870E080E5AB
:1057700090E00E94DF058091140690911506059730
:1057800061F5FEE3EF2EF3E0FF2E01E02FE130E0C4
:105790004FEF5FEF62E370E08FE090E00E949905C9
:1057A000A6E2EA2EA3E0FA2E2FE130E04FEF5FEF02
:1057B00066E470E08FE090E00E949905E090F705C4
:1057C000F090F80503E02FE130E04FEF5FEF62E883
:1057D00070E080E590E00E94DF05809114069091D2
:1057E000150622C2892B61F57EE0E72E73E0F72EC5
:1057F00001E02FE130E04FEF5FEF62E370E08FE018
:1058000090E00E949905E6EFEE2EE2E0FE2E2FE1F9
:1058100030E04FEF5FEF66E470E08FE090E00E94D1
:105820009905E090F905F090FA0503E02FE130E0EA
:105830004FEF5FEF62E870E080E590E00E94DF05E7
:1058400080911406909115068130910531F4809174
:105850006B068F5F80936B062EC0029761F55EE04A
:10586000E52E53E0F52E01E02FE130E04FEF5FEF42
:1058700062E370E08FE090E00E94990566EFE62E0B
:1058800062E0F62E2FE130E04FEF5FEF66E470E06C
:105890008FE090E00E949905E090F905F090FA05FC
:1058A00003E02FE130E04FEF5FEF62E870E080E56A
:1058B00090E00E94DF0580911406909115060497F0
:1058C00061F53EE0E32E33E0F32E01E02FE130E01E
:1058D0004FEF5FEF62E370E08FE090E00E94990588
:1058E00046EFE42E42E0F42E2FE130E04FEF5FEF81
:1058F00066E470E08FE090E00E949905E090F90581
:10590000F090FA0503E02FE130E04FEF5FEF62E83F
:1059100070E080E590E00E94DF0580911406909190
:105920001506059761F59EE0E92E93E0F92E01E05A
:105930002FE130E04FEF5FEF62E370E08FE090E047
:105940000E94990526EFE22E22E0F22E2FE130E0B0
:105950004FEF5FEF66E470E08FE090E00E94990502
:10596000E090F905F090FA0503E02FE130E04FEF09
:105970005FEF62E870E080E590E00E94DF058091D3
:10598000140690911506069709F08AC11EE0E12ED3
:1059900013E0F12E01E02FE130E04FEF5FEF62E323
:1059A00070E08FE090E00E94990586EFE82E82E09B
:1059B000F82E2FE130E04FEF5FEF66E470E08FE00C
:1059C00090E00E949905E090F905F090FA0503E057
:1059D0002FE130E04FEF5FEF62E870E080E590E0AC
:1059E0000E94DF055DC1892BF1F4B6E7EB2EB2E032
:1059F000FB2E01E02FE130E04FEF5FEF6CE370E052
:105A00008FE090E00E949905E0900306F090040674
:105A100003E02FE130E04FEF5FEF62E870E080E5F8
:105A200090E00E94DF058091140690911506019781
:105A300009F058C0A6E7EA2EA2E0FA2E01E02FE115
:105A400030E04FEF5FEF6CE370E08FE090E00E949A
:105A50009905E0900306F090040639C0892BF1F413
:105A6000FCECEF2EF2E0FF2E01E02FE130E04FEFF3
:105A70005FEF6CE370E08FE090E00E949905E090AA
:105A80000506F090060603E02FE130E04FEF5FEFF0
:105A900062E870E080E590E00E94DF0580911406E6
:105AA000909115060197F1F4ECECEE2EE2E0FE2E5B
:105AB00001E02FE130E04FEF5FEF6CE370E08FE04B
:105AC00090E00E949905E0900506F090060603E03C
:105AD0002FE130E04FEF5FEF62E870E080E590E0AB
:105AE0000E94DF0580911406909115068230910581
:105AF00009F49CC09C01245031092230310508F082
:105B000093C094C0892B09F07CC074EEE72E72E03C
:105B1000F72E01E02FE130E04FEF5FEF6CE370E034
:105B20008EE190E00E9499058091FB059091FC0523
:105B3000019779F463E4E62E65E0F62E03E02FE1A9
:105B400030E04FEF5FEF62E870E080E590E00E94A8
:105B500099058091FB059091FC05892B79F45EE312
:105B6000E52E55E0F52E03E02FE130E04FEF5FEF3B
:105B700062E870E080E590E00E9499058091FB0565
:105B80008093DA053EC0892BE1F58091DA05811119
:105B90000AC010926B0643C0892B99F58091DA05F3
:105BA0008111AEC1F6CF8130D1F53EE6E32E33E070
:105BB000F32E01E02FE130E04FEF5FEF62E370E0A2
:105BC0008FE090E00E94990546EBE42E42E0F42E2F
:105BD0002FE130E04FEF5FEF66E470E08FE090E0A0
:105BE0000E949905E090FD05F090FE0503E02FE18D
:105BF00030E04FEF5FEF62E870E080E590E00E94F8
:105C0000DF0580911406909115068130910571F0A1
:105C10008230910559F08430910541F002C080E056
:105C200090E08530910511F00697D1F580916B06D3
:105C30008F5F80936B0634C0009731F09C01215038
:105C400031092230310518F410926B0620C00497F8
:105C5000F1F48FE4E82E82E0F82E01E02FE130E04D
:105C60004FEF5FEF6CE370E08FE090E00E949905EA
:105C7000E0900706F090080603E02FE130E04FEFD8
:105C80005FEF62E870E080E590E00E94DF058091C0
:105C90001406909115060597029710F410926B0662
:105CA00080913A06813009F00EC180937F061092F0
:105CB00047068091140690911506892B41F5E091D5
:105CC0001F06F0912006E830F10508F5EB57FF4F6D
:105CD0004EE150E00C94F13F64E972E014C066E7D5
:105CE00072E011C068E572E00EC06AE372E00BC0BA
:105CF0006CE172E008C06EEF71E005C060EE71E02B
:105D000002C062EC71E08BEE95E00E941943809135
:105D10001406909115060197E1F480911F06909169
:105D200020068130910569F038F0029791F44EE138
:105D300050E068E671E009C04EE150E064EA71E0CD
:105D400004C04EE150E066E871E08BEE95E00E9401
:105D5000194380911406909115060297E1F4809101
:105D60001F06909120068130910569F038F0029766
:105D700091F44EE150E06EE071E009C04EE150E078
:105D80006AE471E004C04EE150E06CE271E08BEE39
:105D900095E00E941943809114069091150604978E
:105DA000E1F480911F06909120068130910569F001
:105DB00038F0029791F44EE150E064EB70E009C0D6
:105DC0004EE150E060EF70E004C04EE150E062ED63
:105DD00070E08BEE95E00E9419438091140690913B
:105DE00015060597E1F480911F06909120068130F9
:105DF000910569F038F0029791F44EE150E06AE5C0
:105E000070E009C04EE150E066E970E004C04EE188
:105E100050E068E770E08BEE95E00E9419438091B6
:105E20001406909115060697E1F480911F06909153
:105E300020068130910569F038F0029791F44EE127
:105E400050E060E070E009C04EE150E06CE370E0CB
:105E500004C04EE150E06EE170E08BEE95E00E94F0
:105E600019438FE190E00E941906809114069091E9
:105E70001506892B09F477D18091140690911506A7
:105E8000019711F40E944F398091140690911506E4
:105E9000029711F40E94563A8091140690911506CB
:105EA000049711F40E945B3B8091140690911506B3
:105EB000059711F40E944C258091140690911506C7
:105EC000069709F448D080913A0681110CC081E010
:105ED00080937F0610924706109209068FE190E0AA
:105EE0000E941906E3D2C0933A062FE788E391E0B7
:105EF000215080409040E1F700C000000C946626DD
:105F0000813009F08CCE9FE9E92E92E0F92E01E074
:105F10002FE130E04FEF5FEF62E370E08FE090E061
:105F20000E9499052CE8E22E22E0F22E2FE130E0CB
:105F30004FEF5FEF66E470E08FE090E00E9499051C
:105F4000E090FF05F090000651CECF911F910F9188
:105F5000FF90EF900895EF92FF920F931F93CF93CE
:105F6000DF93A895809147068111F6C08FE190E0FC
:105F70000E9419060E944F0C80916D0690E090934C
:105F8000200680931F0685E080933A06C1E0D5E0A5
:105F9000809147068111E0C0A8950E94DD0C809198
:105FA0003A068230A9F480911F069091200601964E
:105FB0009093200680931F060FE110E02CE330E061
:105FC00046EE50E069E670E081E090E00E94A404B3
:105FD00080913A068330A9F480911F0690912006A3
:105FE00001979093200680931F060FE110E02CE3A9
:105FF00030E046EE50E069E670E081E090E00E941B
:10600000A40480911F0690912006039720F010921F
:10601000200610921F0680911F0690912006813065
:10602000910589F1D0F0029709F046C081E7E82E8A
:1060300084E0F82E02E02FE130E04FEF5FEF6DE7F4
:1060400070E088E290E00E94990582E080936D06FE
:106050004EE150E060E070E02BC025E8E22E24E045
:10606000F22E02E02FE130E04FEF5FEF6DE770E0DE
:1060700088E290E00E94990510926D064EE150E092
:106080006CE370E015C09BE7E92E94E0F92E02E086
:106090002FE130E04FEF5FEF6DE770E088E290E0D6
:1060A0000E949905C0936D064EE150E06EE170E0EC
:1060B0008BEE95E00E94FC4280913A06811110C05F
:1060C000A895C09347061092260610922506C09305
:1060D00035068FE190E00E941906A8950E943B1FAB
:1060E00080913A06813061F5A89580934706109219
:1060F000260610922506809335068FE190E00E94D7
:106100001906A89510927F0680916D06813069F07E
:1061100038F0823091F44EE150E060E070E009C068
:106120004EE150E06CE370E004C04EE150E06EE1FF
:1061300070E08BEE95E00E94FC42A8950E945226EA
:10614000D0933A062FEF80E792E0215080409040B4
:10615000E1F700C000001CCFDF91CF911F910F919C
:10616000FF90EF900895AF92BF92CF92DF92EF929F
:10617000FF920F931F93CF93DF93A89580914706CB
:10618000811189C18FE190E00E9419060E944F0C95
:106190008091710690E09093200680931F0685E021
:1061A00080933A06E7E0DE2EF6E0CF2ED5E0A4E0BD
:1061B000BA2EB3E0AB2EC1E08091470681116BC1CE
:1061C000A8950E94DD0C80913A068230A9F4809156
:1061D0001F069091200601969093200680931F063B
:1061E0000FE110E02CE330E046EE50E069E670E0AD
:1061F00081E090E00E94A40480913A068330A9F4E3
:1062000080911F069091200601979093200680931D
:106210001F060FE110E02CE330E046EE50E069E6A7
:1062200070E081E090E00E94A40480911F069091AC
:106230002006089720F01092200610921F06E09189
:106240001F06F0912006E830F10508F0BEC0E357C4
:10625000FF4F0C94F13F74E9E72E74E0F72E02E053
:106260002FE130E04FEF5FEF6DE770E082E390E009
:106270000E949905109271064EE150E064E972E0C7
:106280009AC06FE8E62E64E0F62E02E02FE130E0DF
:106290004FEF5FEF6DE770E082E390E00E949905B9
:1062A000C09371064EE150E066E772E084C055E8A5
:1062B000E52E54E0F52E02E02FE130E04FEF5FEFE6
:1062C0006DE770E088E290E00E94990582E080939B
:1062D00071064EE150E068E572E06DC04BE7E42ED8
:1062E00044E0F42E02E02FE130E04FEF5FEF6DE786
:1062F00070E088E290E00E949905A09271064EE15C
:1063000050E06AE372E057C031E7E32E34E0F32E49
:1063100002E02FE130E04FEF5FEF6DE770E088E2E1
:1063200090E00E949905B092710644E150E06CE162
:1063300072E041C027E6E22E24E0F22E02E02FE1D7
:1063400030E04FEF5FEF6DE770E088E290E00E9491
:106350009905D09371064EE150E06EEF71E02BC0CD
:106360009DE5E92E94E0F92E02E02FE130E04FEFB9
:106370005FEF6DE770E088E290E00E949905C092BF
:1063800071064EE150E060EE71E015C083E5E82E45
:1063900084E0F82E02E02FE130E04FEF5FEF6DE791
:1063A00070E088E290E00E949905D09271064EE17B
:1063B00050E062EC71E08BEE95E00E94FC428FE5CC
:1063C0009AEE0197F1F700C0000080913A06811122
:1063D0000FC0A895C0934706109226061092250676
:1063E000C09335068FE190E00E9419060E943B1F82
:1063F00080913A06813009F041C0A8958093470604
:106400001092260610922506809335068FE190E0C3
:106410000E94190610927F06E09171068E2F90E07F
:106420008830910540F5FC01EB56FF4F4EE150E0FE
:106430000C94F13F64E972E014C066E772E011C0A9
:1064400068E572E00EC06AE372E00BC06CE172E0D6
:1064500008C06EEF71E005C060EE71E002C062EC52
:1064600071E08BEE95E00E94FC428FE59AEE019779
:10647000F1F700C00000A8950E945226D0933A067A
:10648000A8959FEF20E782E0915020408040E1F7FF
:1064900000C0000091CEDF91CF911F910F91FF902E
:1064A000EF90DF90CF90BF90AF900895BF92CF92C2
:1064B000DF92EF92FF920F931F93CF93DF93809120
:1064C00009068111E2C68FE190E00E9419060E9440
:1064D000450D10926C0685E080933A0698E5C92E2A
:1064E00092E0D92ECAE5D0E025E0B22E80910906CF
:1064F0008111CBC6E0916B068E2F90E08E30910516
:1065000008F0B2C6FC01E356FF4F0C94F13F1BE2CA
:10651000E12E14E0F12E01E02FE130E04FEF5FEFCC
:1065200062E370E08FE090E00E94990584E2E82E3B
:1065300084E0F82E2FE130E04FEF5FEF66E470E08B
:106540008CE390E00E949905E090EB05F090EC055B
:1065500003E02FE130E040E058EF62E870E080E5D2
:1065600090E00E94DF058091EB059091EC059093FF
:10657000DF058093DE050E94DD0C80913A068230B3
:10658000A9F48091DE059091DF0501969093DF05D7
:106590008093DE050FE110E02CE330E046EE50E0A2
:1065A00069E670E081E090E00E94A40480913A06E0
:1065B0008330A9F48091DE059091DF0501979093D7
:1065C000DF058093DE050FE110E02CE330E046EEBE
:1065D00050E069E670E081E090E00E94A4048091C0
:1065E000DE059091DF058F35914020F01092DF0598
:1065F0001092DE058091DE059091DF059093EC0509
:106600008093EB0528C6ACE0EA2EA4E0FA2E01E068
:106610002FE130E04FEF5FEF62E370E08FE090E05A
:106620000E949905BEEFEB2EB3E0FB2E2FE130E088
:106630004FEF5FEF66E470E08CE390E00E94990515
:10664000E090ED05F090EE0503E02FE130E040E052
:1066500058EF62E870E080E590E00E94DF058091ED
:10666000ED059091EE0590933206809331060E94DD
:10667000DD0C80913A068230A9F480913106909128
:106680003206019690933206809331060FE110E0B6
:106690002CE330E046EE50E069E670E081E090E007
:1066A0000E94A40480913A068330A9F480913106B7
:1066B00090913206019790933206809331060FE154
:1066C00010E02CE330E046EE50E069E670E081E057
:1066D00090E00E94A4048091310690913206853F9B
:1066E000914020F0109232061092310680913106CE
:1066F000909132069093EE058093ED05ACC5E6EEE1
:10670000EE2EE3E0FE2E01E02FE130E04FEF5FEFF1
:1067100062E370E08FE090E00E949905FEECEF2EBE
:10672000F3E0FF2E2FE130E04FEF5FEF66E470E023
:106730008FE090E00E949905E090EF05F090F00561
:1067400003E02FE130E040E058EF62E870E080E5E0
:1067500090E00E94DF058091EF059091F005909305
:106760007A06809379060E94DD0C80913A06823089
:10677000A9F48091790690917A06019690937A0611
:10678000809379060FE110E02CE330E046EE50E014
:1067900069E670E081E090E00E94A40480913A06EE
:1067A0008330A9F48091790690917A0601979093AD
:1067B0007A06809379060FE110E02CE330E046EE94
:1067C00050E069E670E081E090E00E94A4048091CE
:1067D000790690917A064F9730F08FE090E0909391
:1067E0007A06809379068091790690917A060F97C0
:1067F00030F48FE090E090937A0680937906809150
:10680000790690917A069093F0058093EF0523C561
:1068100066EBE62E63E0F62E01E02FE130E04FEF6D
:106820005FEF62E370E08FE090E00E9499057EE9FF
:10683000E72E73E0F72E2FE130E04FEF5FEF66E4D5
:1068400070E08FE090E00E949905E090F105F090F3
:10685000F20503E02FE130E040E058EF62E870E03D
:1068600080E590E00E94DF058091F1059091F205AE
:1068700090931C0680931B060E94DD0C80913A06C3
:106880008230A9F480911B0690911C06019690938A
:106890001C0680931B060FE110E02CE330E046EE6F
:1068A00050E069E670E081E090E00E94A4048091ED
:1068B0003A068330A9F480911B0690911C0601973B
:1068C00090931C0680931B060FE110E02CE330E050
:1068D00046EE50E069E670E081E090E00E94A4049A
:1068E00080911B0690911C064F9730F08FE090E04E
:1068F00090931C0680931B0680911B0690911C06AA
:106900000F9730F48FE090E090931C0680931B0665
:1069100080911B0690911C069093F2058093F105DF
:106920009AC456E8E52E53E0F52E01E02FE130E061
:106930004FEF5FEF6CE370E08FE090E00E9499050D
:106940008091F3059091F405019779F443E4E42EE6
:1069500045E0F42E03E02FE130E040E058EF62E83C
:1069600070E080E590E00E9499058091F305909198
:10697000F405892B79F43EE3E32E35E0F32E03E0B2
:106980002FE130E040E058EF62E870E080E590E011
:106990000E9499058091F305809346060E94DD0CC4
:1069A00080913A06823089F4809146068F5F809309
:1069B00046060FE110E02CE330E046EE50E069E6D9
:1069C00070E081E090E00E94A40480913A06833058
:1069D00089F4809146068150809346060FE110E0CD
:1069E0002CE330E046EE50E069E670E081E090E0B4
:1069F0000E94A40480914606823010F01092460650
:106A00008091460690E09093F4058093F30523C4AB
:106A10009EE6E92E93E0F92E01E02FE130E04FEF02
:106A20005FEF62E370E08FE090E00E94990526E559
:106A3000E22E23E0F22E2FE130E04FEF5FEF66E42D
:106A400070E08FE090E00E949905E090F505F090ED
:106A5000F60503E020E038EF4FEF5FEF62E870E00B
:106A600080E590E00E94DF058091F5059091F605A4
:106A700090931A06809319060E94DD0C80913A06C5
:106A80008230A9F48091190690911A06019690938C
:106A90001A06809319060FE110E02CE330E046EE71
:106AA00050E069E670E081E090E00E94A4048091EB
:106AB0003A068330A9F48091190690911A0601973D
:106AC00090931A06809319060FE110E02CE330E052
:106AD00046EE50E069E670E081E090E00E94A40498
:106AE0008091190690911A068B3F910520F0109223
:106AF0001A06109219068091190690911A06909321
:106B0000F6058093F505A7C31EE3E12E13E0F12EF1
:106B100001E02FE130E04FEF5FEF62E370E08FE0E4
:106B200090E00E94990586E2E82E83E0F82E2FE19E
:106B300030E04FEF5FEF66E470E08FE090E00E949E
:106B40009905E090F705F090F80503E02FE130E0BB
:106B500040E058EF62E870E080E590E00E94DF05D9
:106B60008091F70580932A060E94DD0C80913A06F9
:106B7000823089F480912A068F5F80932A060FE184
:106B800010E02CE330E046EE50E069E670E081E092
:106B900090E00E94A40480913A06833089F48091A9
:106BA0002A06815080932A060FE110E02CE330E0A2
:106BB00046EE50E069E670E081E090E00E94A404B7
:106BC00080912A06853610F010922A0680912A06B6
:106BD00090E09093F8058093F7053DC3AEE0EA2E70
:106BE000A3E0FA2E01E02FE130E04FEF5FEF62E328
:106BF00070E08FE090E00E949905B6EFEB2EB2E0D6
:106C0000FB2E2FE130E04FEF5FEF66E470E08FE0A6
:106C100090E00E949905E090F905F090FA0503E0F4
:106C20002FE130E040E058EF62E870E080E590E06E
:106C30000E94DF058091F905809329060E94DD0CF2
:106C400080913A06823089F4809129068F5F809383
:106C500029060FE110E02CE330E046EE50E069E653
:106C600070E081E090E00E94A40480913A068330B5
:106C700089F4809129068150809329060FE110E064
:106C80002CE330E046EE50E069E670E081E090E011
:106C90000E94A40480912906853610F010922906DE
:106CA0008091290690E09093FA058093F905D3C26C
:106CB000F6E7EF2EF2E0FF2E01E02FE130E04FEF9C
:106CC0005FEF6CE370E08FE090E00E949905E09048
:106CD0000306F090040603E02FE130E040E058EFB7
:106CE00062E870E080E590E00E94DF058091030695
:106CF0009091040690936806809367060E94DD0CCD
:106D000080913A068230A9F48091670690916806D6
:106D1000019690936806809367060FE110E02CE3DC
:106D200030E046EE50E069E670E081E090E00E94DD
:106D3000A40480913A068330A9F48091670690916B
:106D40006806019790936806809367060FE110E04C
:106D50002CE330E046EE50E069E670E081E090E040
:106D60000E94A4048091670690916806893C910571
:106D700020F0D0936806C0936706809167069091D3
:106D800068068A35910520F4D0936806C09367069B
:106D9000809167069091680690930406809303069D
:106DA0005AC2ECECEE2EE2E0FE2E01E02FE130E0E4
:106DB0004FEF5FEF6CE370E08FE090E00E94990589
:106DC000E0900506F090060603E02FE130E040E099
:106DD00058EF62E870E080E590E00E94DF05809166
:106DE0000506909106069093EA058093E9050E94B6
:106DF000DD0C80913A068230A9F48091E9059091EA
:106E0000EA0501969093EA058093E9050FE110E009
:106E10002CE330E046EE50E069E670E081E090E07F
:106E20000E94A40480913A068330A9F48091E90578
:106E30009091EA0501979093EA058093E9050FE1A7
:106E400010E02CE330E046EE50E069E670E081E0CF
:106E500090E00E94A4048091E9059091EA05C3970F
:106E600020F01092EA051092E9058091E9059091D1
:106E7000EA059093060680930506EDC174EEE72EB1
:106E800072E0F72E01E02FE130E04FEF5FEF6CE3AF
:106E900070E08EE190E00E9499058091FB05909151
:106EA000FC05019779F463E4E62E65E0F62E03E035
:106EB0002FE130E040E058EF62E870E080E590E0DC
:106EC0000E9499058091FB059091FC05892B79F42E
:106ED0005EE3E52E55E0F52E03E02FE130E040E0E3
:106EE00058EF62E870E080E590E00E94990580919B
:106EF000FB058093DA050E94DD0C80913A06823012
:106F000089F48091DA058F5F8093DA050FE110E054
:106F10002CE330E046EE50E069E670E081E090E07E
:106F20000E94A40480913A06833089F48091DA05A6
:106F300081508093DA050FE110E02CE330E046EE5B
:106F400050E069E670E081E090E00E94A404809146
:106F5000DA05823010F01092DA058091DA0590E0BF
:106F60009093FC058093FB0576C18091DA05811131
:106F700003C010926B0678C1813009F075C13EE6FE
:106F8000E32E33E0F32E01E02FE130E04FEF5FEF2F
:106F900062E370E08FE090E00E94990546EBE42EFA
:106FA00042E0F42E2FE130E04FEF5FEF66E470E057
:106FB0008FE090E00E949905E090FD05F090FE05BD
:106FC00003E02FE130E040E058EF62E870E080E558
:106FD00090E00E94DF058091FD059091FE05909361
:106FE0006A06809369060E94DD0C80913A06823021
:106FF000A9F48091690690916A06019690936A06B9
:10700000809369060FE110E02CE330E046EE50E09B
:1070100069E670E081E090E00E94A40480913A0665
:107020008330A9F48091690690916A060197909344
:107030006A06809369060FE110E02CE330E046EE2B
:1070400050E069E670E081E090E00E94A404809145
:10705000690690916A068B3F910520F010926A06AE
:10706000109269068091690690916A069093FE05D8
:107070008093FD05F0C08091DA05882309F479CF6B
:10708000813009F0F1C09FE9E92E92E0F92E01E08C
:107090002FE130E04FEF5FEF62E370E08FE090E0D0
:1070A0000E9499052CE8E22E22E0F22E2FE130E03A
:1070B0004FEF5FEF66E470E08FE090E00E9499058B
:1070C000E090FF05F090000603E02FE130E040E0A3
:1070D00058EF62E870E080E590E00E94DF05809163
:1070E000FF059091000690934506809344060E9408
:1070F000DD0C80913A068230A9F48091440690918B
:107100004506019690934506809344060FE110E0F2
:107110002CE330E046EE50E069E670E081E090E07C
:107120000E94A40480913A068330A9F48091440619
:1071300090914506019790934506809344060FE190
:1071400010E02CE330E046EE50E069E670E081E0CC
:1071500090E00E94A4048091440690914506C39754
:1071600020F01092450610924406809144069091BA
:107170004506909300068093FF056DC08FE4E82ECE
:1071800082E0F82E01E02FE130E04FEF5FEF6CE39B
:1071900070E08FE090E00E949905E0900706F09083
:1071A000080603E02FE130E040E058EF62E870E0CD
:1071B00080E590E00E94DF05809107069091080627
:1071C00090930F0680930E060E94DD0C80913A0684
:1071D0008230A9F480910E0690910F06019690934B
:1071E0000F0680930E060FE110E02CE330E046EE30
:1071F00050E069E670E081E090E00E94A404809194
:107200003A068330A9F480910E0690910F060197FB
:1072100090930F0680930E060FE110E02CE330E010
:1072200046EE50E069E670E081E090E00E94A40440
:107230008091E9059091EA058935924020F0D0923D
:107240000F06C0920E0680910E0690910F06909345
:107250000806809307068FE798E321E0815090406D
:107260002040E1F700C0000080913A06813051F4DF
:107270008093090610927F068FE190E00E94190624
:107280000E945226B0923A0631C9DF91CF911F91E8
:107290000F91FF90EF90DF90CF90BF900895EF9205
:1072A000FF920F931F93CF93DF93A895809147068A
:1072B0008111F5C08FE190E00E9419060E944F0CE9
:1072C00080911D0690E09093200680931F0685E034
:1072D00080933A06C1E0D5E0809147068111DFC076
:1072E000A8950E94DD0C80913A068230A9F4809125
:1072F0001F069091200601969093200680931F060A
:107300000FE110E02CE330E046EE50E069E670E07B
:1073100081E090E00E94A40480913A068330A9F4B1
:1073200080911F06909120060197909320068093EC
:107330001F060FE110E02CE330E046EE50E069E676
:1073400070E081E090E00E94A40480911F0690917B
:107350002006039720F01092200610921F06A89591
:1073600080911F06909120068130910589F1D0F01F
:10737000029709F046C081E7E82E84E0F82E02E08B
:107380002FE130E04FEF5FEF6DE770E088E290E0D3
:107390000E94990582E080931D064EE150E068E668
:1073A00071E02BC025E8E22E24E0F22E02E02FE16E
:1073B00030E04FEF5FEF6DE770E088E290E00E9411
:1073C000990510921D064EE150E064EA71E015C087
:1073D0009BE7E92E94E0F92E02E02FE130E04FEF39
:1073E0005FEF6DE770E088E290E00E949905C0933E
:1073F0001D064EE150E066E871E08BEE95E00E94DC
:10740000FC4280913A0681110FC0A895C0934706AF
:107410001092260610922506C09335068FE190E063
:107420000E9419060E943B1F80913A06813059F54F
:10743000A895809347061092260610922506809301
:1074400035068FE190E00E94190610927F06809128
:107450001D06813069F038F0823091F44EE150E041
:1074600068E671E009C04EE150E064EA71E004C0F2
:107470004EE150E066E871E08BEE95E00E94FC4240
:10748000A8950E945226D0933A062FEF80E792E00B
:10749000215080409040E1F700C000001DCFDF91F7
:1074A000CF911F910F91FF90EF900895EF92FF926F
:1074B0000F931F93CF93DF93A89580914706811177
:1074C000F3C08FE190E00E9419060E944F0C80915A
:1074D000240690E09093200680931F0685E0809319
:1074E0003A06C1E0D5E0809147068111DDC0A8953C
:1074F0000E94DD0C80913A068230A9F480911F062B
:107500009091200601969093200680931F060FE12C
:1075100010E02CE330E046EE50E069E670E081E0F8
:1075200090E00E94A40480913A068330A9F48091EF
:107530001F069091200601979093200680931F06C6
:107540000FE110E02CE330E046EE50E069E670E039
:1075500081E090E00E94A40480911F069091200693
:10756000039720F01092200610921F0680911F06AC
:10757000909120068130910589F1D0F0029709F0B1
:1075800045C081E7E82E84E0F82E02E02FE130E0EC
:107590004FEF5FEF6DE770E088E290E00E949905A1
:1075A00082E0809324064EE150E06EE071E02BC053
:1075B00025E8E22E24E0F22E02E02FE130E04FEF4A
:1075C0005FEF6DE770E088E290E00E94990510920D
:1075D00024064EE150E06AE471E015C09BE7E92E15
:1075E00094E0F92E02E02FE130E04FEF5FEF6DE71E
:1075F00070E088E290E00E949905C09324064EE175
:1076000050E06CE271E08BEE95E0F6D780913A069F
:10761000811110C0A895C0934706109226061092BB
:107620002506C09335068FE190E00E941906A895C3
:107630000E943B1F80913A06813051F5A8958093B6
:1076400047061092260610922506809335068FE194
:1076500090E00E94190610927F06809124068130E6
:1076600069F038F0823089F44EE150E06EE071E06C
:1076700009C04EE150E06AE471E004C04EE150E020
:107680006CE271E08BEE95E0B7D7A8950E94522688
:10769000D0933A062FEF80E792E02150804090404F
:1076A000E1F700C000001FCFDF91CF911F910F9134
:1076B000FF90EF900895EF92FF920F931F93CF9357
:1076C000DF93A895809147068111F4C08FE190E087
:1076D0000E9419060E944F0C80917C0690E09093C6
:1076E000200680931F0685E080933A06C1E0D5E02E
:1076F000809147068111DEC0A8950E94DD0C809123
:107700003A068230A9F480911F06909120060196D6
:107710009093200680931F060FE110E02CE330E0E9
:1077200046EE50E069E670E081E090E00E94A4043B
:1077300080913A068330A9F480911F06909120062B
:1077400001979093200680931F060FE110E02CE331
:1077500030E046EE50E069E670E081E090E00E94A3
:10776000A40480911F0690912006039720F01092A8
:10777000200610921F0680911F06909120068130EE
:10778000910589F1D0F0029709F045C081E7E82E14
:1077900084E0F82E02E02FE130E04FEF5FEF6DE77D
:1077A00070E088E290E00E94990582E080937C0678
:1077B0004EE150E064EB70E02BC025E8E22E24E0BF
:1077C000F22E02E02FE130E04FEF5FEF6DE770E067
:1077D00088E290E00E94990510927C064EE150E00C
:1077E00060EF70E015C09BE7E92E94E0F92E02E00F
:1077F0002FE130E04FEF5FEF6DE770E088E290E05F
:107800000E949905C0937C064EE150E062ED70E065
:107810008BEE95E0F1D680913A06811110C0A895C3
:10782000C09347061092260610922506C09335068F
:107830008FE190E00E941906A8950E943B1F80915D
:107840003A06813059F5A89580934706109226068E
:1078500010922506809335068FE190E00E9419066C
:10786000A89510927F0680917C06813069F038F0EF
:10787000823089F44EE150E064EB70E009C04EE1E3
:1078800050E060EF70E004C04EE150E062ED70E067
:107890008BEE95E0B1D6A8950E945226D0933A0679
:1078A0002FEF80E792E0215080409040E1F700C048
:1078B00000001ECFDF91CF911F910F91FF90EF90AD
:1078C00008950F931F938091120690911306892BB0
:1078D00009F099C0809173069091740683359105E3
:1078E000A9F581E090E090931306809312060E9420
:1078F00087130FE110E02CE330E044E650E06BE446
:1079000070E08EE690E00E94A40424E230E04AE5B4
:1079100050E064E670E088E090E00E94A40424E275
:1079200030E04AE550E064E670E088E090E00E94D4
:10793000A40424E230E04AE550E064E670E08FED14
:1079400090E00E94A4040E943B1FA8950E94101E74
:107950000E94F119A89503E02FE130E04FEF5FEFAF
:1079600069E170E085E890E00E9404110E94BE1D6C
:107970000E949C108091120690911306019781F548
:10798000A8950E9487130FE110E02CE330E044E655
:1079900050E06BE470E08EE690E00E94A40424E2E4
:1079A00030E04AE550E064E670E088E090E00E9454
:1079B000A40424E230E04AE550E064E670E088E0A8
:1079C00090E00E94A40424E230E04AE550E064E63E
:1079D00070E08FED90E00E94A4040E943B1FA895E8
:1079E0002FEF81EE94E0215080409040E1F700C0FD
:1079F00000000E94D20E0E94E71D0E94580F1F91A6
:107A00000F910C94C80F1F910F9108951F920F9220
:107A10000FB60F9211248F939F938CB190E09093A7
:107A20007406809373069F918F910F900FBE0F90F5
:107A30001F9018951F920F920FB60F9211242F933B
:107A40008F939F938091E5059091E6050196883E7E
:107A500023E0920728F49093E6058093E50504C09F
:107A60001092E6051092E50580911006811105C07F
:107A700010927606109275060BC0813049F4809101
:107A8000750690917606019690937606809375061A
:107A900080912F06811105C01092E4051092E30534
:107AA0000BC0813049F48091E3059091E405019683
:107AB0009093E4058093E30580912706811105C02A
:107AC0001092E8051092E7050BC0813049F48091CF
:107AD000E7059091E80501969093E8058093E70506
:107AE0009F918F912F910F900FBE0F901F9018951F
:107AF0002FEF89E698E1215080409040E1F700C0E7
:107B000000008FEF8ABB81BB8093610081E084BB62
:107B100088EA8FBD8CE08EBD1DBC1CBC17BC16BC9A
:107B20008AE78BBD82E18ABD19BC18BC109279002E
:107B30001092780080E187BF10BE87E683BF12BE37
:107B400011BE81E880938B0085E080938A001092BB
:107B5000890010928800109281001092800010928B
:107B60008700109286001092850010928400109277
:107B70008300109282001BB888E98AB986E080935E
:107B80009500109290008FE289B98FE181BD8FE05E
:107B900081BD77D081E00E94B0038FE190E00E9428
:107BA000190681E090E090931306809312061092DC
:107BB00026061092250610921506109214061092B1
:107BC000E6051092E50510922C0610922B061092F5
:107BD000E205109211061092770610920A0680E5CF
:107BE00090E09093740680937306809164008E7F7A
:107BF000809364008091650081608093650080912E
:107C00006400886080936400809165008860809340
:107C100065007894A49AAC9A2FEF85EA9EE02150F3
:107C200080409040E1F700C00000A895AC9882EB3E
:107C300092E0F2D4813079F00E94301AA8950E9427
:107C40009D1DA89561E083EB92E0FCD4A89561E0CE
:107C500082EB92E0F7D4A8958091120690911306DA
:107C6000019721F4A8950E943B1FA895A89529DEAD
:107C7000F2CFC098AB9AAF9A8FB9779BFECF8FB1F6
:107C8000089587E087BBC09AAB9AAF9A83E58DB918
:107C90001EB880E8EEDF80E0ECDF80E0EADF8AE11A
:107CA0008A95F1F700C00895EF92FF920F931F930A
:107CB000CF93DF9300D000D0CDB7DEB77C018B012E
:107CC000A895AB9AAF9A1C821B821A82198280ED0A
:107CD000D0DF80E0CEDF8FB190E09C838B838B81FF
:107CE0009C81982F88279C838B8380E0C2DF2FB1F3
:107CF0008B819C81822B9C838B838B819C8133E045
:107D0000969587953A95E1F79C838B8387EC90E075
:107D10000197F1F700C0000080E9ABDF80E0A9DF48
:107D20008FB190E09A83898389819A81982F8827DF
:107D30009A83898380E09DDF2FB189819A81822B8C
:107D40009A83898389819A8153E0969587955A957C
:107D5000E1F79A8389838B819C81F70191838083EA
:107D600089819A81F801918380830F900F900F9001
:107D70000F90DF91CF911F910F91FF90EF90089599
:107D800070D088F09F5790F0B92F9927B751A0F085
:107D9000D1F0660F771F881F991F1AF0BA95C9F79F
:107DA00012C0B13081F077D0B1E0089574C0672F70
:107DB000782F8827B85F39F0B93FCCF3869577954F
:107DC0006795B395D9F73EF4909580957095619538
:107DD0007F4F8F4F9F4F0895E89409C097FB3EF463
:107DE00090958095709561957F4F8F4F9F4F992308
:107DF000A9F0F92F96E9BB279395F6958795779586
:107E00006795B795F111F8CFFAF4BB0F11F460FF45
:107E10001BC06F5F7F4F8F4F9F4F16C0882311F09D
:107E200096E911C0772321F09EE8872F762F05C0B1
:107E3000662371F096E8862F70E060E02AF09A954C
:107E4000660F771F881FDAF7880F9695879597F941
:107E5000089557FD9058440F551F59F05F3F71F03A
:107E60004795880F97FB991F61F09F3F79F08795A1
:107E70000895121613061406551FF2CF4695F1DF2A
:107E800008C0161617061806991FF1CF86957105BA
:107E9000610508940895E894BB2766277727CB01EE
:107EA00097F908950BD078C069D028F06ED018F0FB
:107EB000952309F05AC05FC01124EECFCADFA0F3AA
:107EC000959FD1F3950F50E0551F629FF001729F6F
:107ED000BB27F00DB11D639FAA27F00DB11DAA1F8E
:107EE000649F6627B00DA11D661F829F2227B00DDB
:107EF000A11D621F739FB00DA11D621F839FA00D66
:107F0000611D221F749F3327A00D611D231F849FB5
:107F1000600D211D822F762F6A2F11249F5750400C
:107F20008AF0E1F088234AF0EE0FFF1FBB1F661FA7
:107F3000771F881F91505040A9F79E3F510570F060
:107F400014C0AACF5F3FECF3983EDCF3869577959B
:107F50006795B795F795E7959F5FC1F7FE2B880F5B
:107F6000911D9695879597F9089597F99F6780E8F1
:107F700070E060E008959FEF80EC089500240A947B
:107F80001616170618060906089500240A941216F4
:107F90001306140605060895092E0394000C11F427
:107FA000882352F0BB0F40F4BF2B11F460FF04C0D4
:107FB0006F5F7F4F8F4F9F4F0895AA1BBB1B51E1EF
:107FC00007C0AA1FBB1FA617B70710F0A61BB70B49
:107FD000881F991F5A95A9F780959095BC01CD01EE
:107FE0000895EE0FFF1F0024001C0BBE0790F691B2
:107FF000E02D0994A29FB001B39FC001A39F700D13
:10800000811D1124911DB29F700D811D1124911DA0
:108010000895BB274A3031F4992322F4BDE29095AC
:1080200081959F4F01C0BB27FB015527AA27880FC9
:10803000991FAA1FA41710F0A41B83955051B9F7DC
:10804000A05DAA3308F0A95DA193009779F7B1115B
:10805000B1931192CB0126C2CF93DF93CDB7DEB798
:10806000AE014B5F5F4FFA0161917191AF01809159
:1080700082069091830603D0DF91CF9108952F92CD
:108080003F924F925F926F927F928F929F92AF92A8
:10809000BF92CF92DF92EF92FF920F931F93CF93F5
:1080A000DF93CDB7DEB72B970FB6F894DEBF0FBEC8
:1080B000CDBF6C017B018A01FC011782168283818E
:1080C00081FFBFC1CE0101963C01F6019381F7010A
:1080D00093FD859193FF81917F01882309F4ADC1C0
:1080E000853239F493FD859193FF81917F0185322B
:1080F00021F4B60190E0E6D1E8CF912C212C312C6F
:10810000FFE1F315D8F08B3279F038F4803279F052
:108110008332A1F4232D20611DC08D3261F08033A4
:1081200069F4232D216016C0832D8260382EE32D43
:10813000E4603E2E2AC0F32DF8601DC037FC2DC030
:1081400020ED280F2A3040F08E32B9F436FC75C18C
:10815000232D2064322E19C036FE06C08AE0989E78
:10816000200D1124922E11C0EAE02E9E200D112424
:10817000222EF32DF0623F2E08C08C3621F4832D81
:108180008068382E02C0883641F4F70193FD85914E
:1081900093FF81917F018111B3CF982F9F7D9554DB
:1081A000933028F40C5F1F4F9FE399830DC08336F3
:1081B00031F0833771F0833509F055C020C0F801E4
:1081C000808189830E5F1F4F88248394912C5301F3
:1081D00012C02801F2E04F0E511CF801A080B180BE
:1081E00036FE03C0692D70E002C06FEF7FEFC5015E
:1081F0004ED14C018201F32DFF773F2E15C028018F
:1082000022E0420E511CF801A080B18036FE03C06E
:10821000692D70E002C06FEF7FEFC5012DD14C01D9
:10822000F32DF0683F2E820133FC19C0822D90E0BF
:1082300088169906A0F4B60180E290E043D12A9412
:10824000F5CFF50137FC859137FE81915F01B601CD
:1082500090E038D121102A9421E0821A91088114EB
:10826000910479F7E1C0843611F0893639F5F801C7
:1082700037FE07C060817181828193810C5F1F4F3F
:1082800008C060817181072E000C880B990B0E5F6E
:108290001F4FF32DFF763F2E97FF09C090958095D5
:1082A000709561957F4F8F4F9F4FF0683F2E2AE06A
:1082B00030E0A30143D1882E861844C0853731F4BD
:1082C000232D2F7EB22E2AE030E025C0932D997FFA
:1082D000B92E8F36C1F018F4883579F0AEC08037EA
:1082E00019F0883721F0A9C0E92FE061BE2EB4FE55
:1082F0000DC0FB2DF460BF2E09C034FE0AC0292F2B
:108300002660B22E06C028E030E005C020E130E053
:1083100002C020E132E0F801B7FE07C06081718140
:10832000828193810C5F1F4F06C06081718180E064
:1083300090E00E5F1F4FA30101D1882E8618FB2D00
:10834000FF773F2E36FE0DC0232D2E7FA22E8914DF
:1083500058F434FE0BC032FC09C0832D8E7EA82E4B
:1083600005C0B82CA32C03C0B82C01C0B92CA4FEA6
:108370000FC0FE01E80DF11D8081803321F49A2D9C
:10838000997EA92E09C0A2FE06C0B394B39404C07E
:108390008A2D867809F0B394A3FC10C0A0FE06C015
:1083A000B21480F4280C922C9B180DC0B21458F40F
:1083B000B60180E290E086D0B394F8CFB21418F4FE
:1083C0002B1802C0982C212CA4FE0FC0B60180E30C
:1083D00090E078D0A2FE16C0A1FC03C088E790E030
:1083E00002C088E590E0B6010CC08A2D867851F075
:1083F000A1FE02C08BE201C080E2A7FC8DE2B601C3
:1084000090E060D0891430F4B60180E390E05AD057
:108410009A94F8CF8A94F301E80DF11D8081B6019A
:1084200090E050D08110F6CF222009F44ECEB60154
:1084300080E290E047D02A94F7CFF60186819781B9
:1084400002C08FEF9FEF2B960FB6F894DEBF0FBEE2
:10845000CDBFDF91CF911F910F91FF90EF90DF90F3
:10846000CF90BF90AF909F908F907F906F905F90D4
:108470004F903F902F900895FC01059061507040FF
:108480000110D8F7809590958E0F9F1F0895FC01DD
:108490006150704001900110D8F7809590958E0F33
:1084A0009F1F0895DC01FC01672F71917723E1F78D
:1084B000329704C07C916D9370836291AE17BF07B1
:1084C000C8F308950F931F93CF93DF93FB0123818C
:1084D00021FD03C08FEF9FEF2CC022FF16C0468105
:1084E0005781248135814217530744F4A081B1811B
:1084F0009D012F5F3F4F318320838C9326813781ED
:108500002F5F3F4F3783268314C08B01EC01FB01A3
:108510000084F185E02D0995892BE1F6D8011696A6
:108520008D919C911797019617969C938E93169711
:10853000CE01DF91CF911F910F910895FA01AA27E3
:10854000283051F1203181F1E8946F936E7F6E5F96
:108550007F4F8F4F9F4FAF4FB1E03ED0B4E03CD044
:10856000670F781F891F9A1FA11D680F791F8A1F27
:10857000911DA11D6A0F711D811D911DA11D20D08E
:1085800009F468943F912AE0269F11243019305D48
:108590003193DEF6CF010895462F4770405D419339
:1085A000B3E00FD0C9F7F6CF462F4F70405D4A3386
:1085B00018F0495D31FD4052419302D0A9F7EACF4E
:1085C000B4E0A6959795879577956795BA95C9F77D
:1085D00000976105710508959B01AC010A2E069470
:1085E0005795479537952795BA95C9F7620F731F29
:1085F000841F951FA01D0895DC01CB01FC01E199AA
:10860000FECF06C0FFBBEEBBE09A31960DB20D92D5
:1086100041505040B8F70895E199FECF9FBB8EBB03
:10862000E09A99278DB30895A8E1B0E042E050E0C8
:10863000E5CFDC01CB0102C02D9105D04150504067
:10864000D8F70895262FE199FECF9FBB8EBB2DBB97
:108650000FB6F894E29AE19A0FBE01960895F2DF00
:08866000272FF1CFF894FFCFA2
:108668000000000200000000DE0700000000575470
:108678003D2025750A47530047533D2025750A5369
:108688004E00534E3D2025750A454E4400574B3D3C
:108698002025750A565000503D332E360A52005296
:1086A8004C3D2025750A68004F3D73740A530047F6
:1086B8003D73740A530053523D53746174696F6E6D
:1086C800200A57500057503D536E36332F506233AF
:1086D800370A57540057503D536E41670A575400A4
:1086E80057503D50726F66696C65300A5754005791
:1086F800503D50726F66696C65310A575400575087
:108708003D50726F66696C65320A57540057503D88
:1087180050726F66696C65330A57540057503D5064
:10872800726F66696C65340A57540057503D507231
:108738006F66696C65350A57540053523D55506849
:108748006561746572200A57500053523D50726536
:10875800686561746572200A57500053523D4D6137
:108768006E75616C200A57500053523D5265626F16
:108778006C6C696E67200A57500053523D43686914
:108788007068656174696E67200A57500053523DDE
:1087980050434268656174696E67200A57500053F8
:1087A800523D5043200A57500056312E307A00204F
:1087B8002020C2F0E5ECFF20F0E5E1EEEBEBE8ED80
:1087C800E3E02020202000C2FBE1E5F0E8F2E5200C
:1087D800F0E5E6E8EC00D2E5ECEFE5F0E0F2F3F0E6
:1087E800E020EFEEEBEEF7EAE8202000EDE8E7E026
:1087F80020EFF0E820E4EEEDE0E3F0E5E2E500D27A
:10880800E5ECEFE5F0E0F2F3F0E020F3E2E5EBE889
:10881800F7E5EDE8FF00202020202020E4EEEDE041
:10882800E3F0E5E2E020202020202000C4EBE8F27D
:10883800E5EBFCEDEEF1F2FC20E2EFE8F2FBE2E022
:10884800EDE8FF00D4F3EDEAF6E8FF20E4EEEDEE04
:10885800E3F0E5E2E000EDE8E6EDE5E3EE20EDE04B
:10886800E3F0E5E2E0F2E5EBFF2020202000CCE099
:10887800EAF1E8ECE0EBFCEDE0FF20ECEEF9EDEEE0
:10888800F1F2FC202000E2E5F0F5EDE5E3EE20ED65
:10889800E0E3F0E5E2E0F2E5EBFF20202000CCE0A9
:1088A800EAF1E8ECE0EBFCEDE0FF20ECEEF9EDEEB0
:1088B800F1F2FC202000E2E5F0F5EDE5E3EE20ED35
:1088C800E0E3F0E5E2E0F2E5EBFF20202000D2E56E
:1088D800ECEFE5F0E0F2F3F0E020E2EAEBFEF7E59A
:1088E800EDE8FF202000CAEEEDF2F0EEEBFC20EF01
:1088F800EE20E2E5F0F5F320202020202000EDE82E
:10890800E6EDE5E3EE20EDE0E3F0E5E2E0F2E5EBAD
:10891800FF2020202000CAEEFDF4F4E8F6E8E5ED9B
:10892800F220EFF0EEF4E8EBFF2020202000E2E553
:10893800F0F5EDE5E3EE20EDE0E3F0E5E2E0F2E569
:10894800EBFF20202000CAEEFDF4F4E8F6E8E5EDA0
:10895800F220EFF0EEF4E8EBFF2020202000EDE01D
:10896800E3F0E5E2E0F2E5EBFF202000D2E5ECEFF2
:10897800E5F0E0F2F3F0E020EDE8E6EDE5E3EE20E7
:1089880020202000EFE0E9EAE82000D2E5ECEFE55E
:10899800F0E0F2F3F0E020ECE5F1F2E02020202016
:1089A8002000C2FBE1E5F0E8F2E520EFF0EEF4E8A4
:1089B800EBFC00CFF0EEF4E8EBFC203500CFF0EE56
:1089C800F4E8EBFC203400CFF0EEF4E8EBFC2033C5
:1089D80000CFF0EEF4E8EBFC203200CFF0EEF4E844
:1089E800EBFC203100CFF0EEF4E8EBFC2030005334
:1089F8006E416700536E506200CAEEECEFFCFEF267
:108A0800E5F000C4EEEF2E20EDE0F1F2F0EEE9EA39
:108A1800E800EFEBE0F20020D1F3F8EAE020EFEB1A
:108A2800E0F22000ECE8EAF0EEF1F5E5EC00D1F335
:108A3800F8EAE000D0E5E1EEEBEBE8EDE32000D06A
:108A4800F3F7EDEEE9002020D0F3F7EDEEE9202072
:108A58002000CDE8E6EDE8E920EDE0E3F02E200087
:108A6800C2E5F0F5EDE8E920EDE0E3F02E00202086
:108A7800D1F2E0EDF6E8FF00E2E5F0F5E000EDE820
:108A8800E7E000CCEEF9EDEEF1F2FC00CFF0E8ED16
:108A9800FFF2EE202000C2DBC1D0C0D2DC00C2DB76
:108AA800CACB00C2CACB00CDE0F1F2F0EEE8F2FC8E
:108AB80000C7E2F3EAEEE2FBE520F1E8E3EDE0EBE4
:108AC800FB00CFF0E5E4F3F1F2E0EDEEE2EAE800D6
:108AD800D3ECEEEBF7E0EDE8FF00C2F0E5ECFF20A9
:108AE800EFE0E9EAE80020C4E0F2F7E8EA20EDE880
:108AF800E62E20EDE0E3F0E5E2E0F2E5EBFF002012
:108B0800C4E0F2F7E8EA20ECE5F1F2E020EFE0E972
:108B1800EAE800F0F3F7EDEEE900EDE8E6EDE8E964
:108B280000EDE0E3F02E00C2E5F0F5EDE8E900C263
:068B3800DBD5CEC40000F5
:00000001FF
